:10000000F9EF24F0FFFFFFFF00C0ECF3E9CF2EF380
:10001000EACF2FF3E1CF30F3E2CF31F3C20ED76E48
:10002000F70ED66E200EF26E8C7E154A162A800EC2
:100030001618006E800E1818005C02E11750155C4F
:1000400004E3010E196E156A166A2EC3E9FF2FC369
:10005000EAFF30C3E1FF31C3E2FFECC300F011005F
:10006000280E0301B66F6E0EB76F750EB86F6C0E6B
:10007000B96F6C0EBA6F290EBB6FBC6BC46BC56BCE
:10008000C26BC36B0301B1C300F0B2C301F0B3C3D1
:1000900002F0010EB127000EB223B32300C0F6FF19
:1000A00001C0F7FF02C0F8FF0900F5CF00F000C063
:1000B000BFF30052D8B470EF11F0BF51250A0BE026
:1000C000AFC3E1FFB0C3E2FFBFC3E6FFAF4BB02B4E
:1000D000C44BC52BD7D7C06BC16BC26BC36B0301BD
:1000E00023D0C287010EB127000EB223B3235AD00A
:1000F000C281010EB127000EB223B32353D0C283B5
:10010000010EB127000EB223B3234CD0C387010EDA
:10011000B127000EB223B32345D0C285010EB1270B
:10012000000EB223B3233ED00301B1C3F6FFB2C326
:10013000F7FFB3C3F8FF0900F5CFD0F3D0512D0A74
:10014000D0E0B1C3F6FFB2C3F7FFB3C3F8FF0900B5
:10015000F5CFD0F3D051200ACBE0B1C3F6FFB2C344
:10016000F7FFB3C3F8FF0900F5CFD0F3D0512B0A46
:10017000C6E0B1C3F6FFB2C3F7FFB3C3F8FF09008F
:10018000F5CFD0F3D051230AC1E0B1C3F6FFB2C31B
:10019000F7FFB3C3F8FF0900F5CFD0F3D051300A11
:1001A000BCE001D09CD70301C2B3C291C2B7C295D3
:1001B000B1C3F6FFB2C3F7FFB3C3F8FF0900F5CF31
:1001C00000F0000E016E00C0D8F337EC3BF0005297
:1001D00038E00301C06BC16BC0C300F0C1C301F0C4
:1001E0000A0E046E000E056E45EC37F0B1C3F6FF43
:1001F000B2C3F7FFB3C3F8FF0900F5CFD0F3030193
:10020000D0510024C06F000E0120C16F300EC05FBE
:10021000000EC15B010EB127000EB223B323B1C3A0
:10022000F6FFB2C3F7FFB3C3F8FF0900F5CF00F044
:10023000000E016E00C0D8F337EC3BF00052CCE169
:1002400036D0B1C3F6FFB2C3F7FFB3C3F8FF09005E
:10025000F5CFD0F30301D0512A0A29E1B4C3E9FF55
:10026000B5C3EAFFEECF00F0EECF01F000C0E9FF2A
:1002700001C0EAFFEECFC0F3EECFC1F3B4C3E9FF94
:10028000B5C3EAFFEECF00F0EECF01F0020E00267C
:10029000000E0122B4C3E1FFB5C3E2FF00C0E6FFD8
:1002A00001C0E6FF010EB127000EB223B323030104
:1002B000B1C3F6FFB2C3F7FFB3C3F8FF0900F5CF30
:1002C000D0F3D0512E0A74E1010EB127000EB223F3
:1002D000B323B1C3F6FFB2C3F7FFB3C3F8FF0900FE
:1002E000F5CFD0F3D0512A0A2AE1B4C3E9FFB5C350
:1002F000EAFFEECF00F0EECF01F000C0E9FF01C051
:10030000EAFFEECFBDF3EECFBEF3B4C3E9FFB5C352
:10031000EAFFEECF00F0EECF01F0020E0026000E55
:100320000122B4C3E1FFB5C3E2FF00C0E6FF01C094
:10033000E6FF010EB127000EB223B32337D0BD6B09
:10034000BE6BB1C3F6FFB2C3F7FFB3C3F8FF09003A
:10035000F5CF00F0000E016E00C0D8F337EC3BF093
:10036000005224E0BDC300F0BEC301F00A0E046ECB
:10037000000E056E45EC37F0B1C3F6FFB2C3F7FFD0
:10038000B3C3F8FF0900F5CFD0F30301D051002427
:10039000BD6F000E0120BE6F300EBD5F000EBE5B54
:1003A000010EB127000EB223B323CBD7030104D033
:1003B0000301BD6BBE6BC3890301B1C300F0B2C3BF
:1003C00001F0B3C302F0010EB127000EB223B32334
:1003D00000C0F6FF01C0F7FF02C0F8FF0900F5CF2B
:1003E000BFF3EDD0C4C300F0C5C301F01200C28951
:1003F000E3D7C3851FD1C28BC3811CD1C3831AD15C
:10040000C28D18D117D1C28BC28F14D1B4C3E9FFEA
:10041000B5C3EAFFEECF00F0EECF01F000C0E9FF78
:1004200001C0EAFFEECFCCF3EECFCDF3B4C3E9FFCA
:10043000B5C3EAFFEECF00F0EECF01F0020E0026CA
:10044000000E0122B4C3E1FFB5C3E2FF00C0E6FF26
:1004500001C0E6FF000ECD1902E1000ECC1904E147
:10046000B60ECC6F030ECD6F0301CE6BCF6BCE51AA
:10047000CC25E96ECF51CD21EA6EEECF00F00052CF
:1004800003E0CE4BCF2BF3D7BD51BE110AE0CF51C5
:10049000BE5D02E1CE51BD5D04E2BDC3CEF3BEC37D
:1004A000CFF30301C151CF5D02E1C051CE5D05E242
:1004B000CE51C05FCF51C15B03D00301C06BC16B94
:1004C000C2B716D0C0C300F0C1C301F0010EC05FB7
:1004D000000EC15B005001100BE0AFC3E1FFB0C3E1
:1004E000E2FF200EE66EAF4BB02BC44BC52BEAD714
:1004F000CEC300F0CFC301F0010ECE5F000ECF5B84
:100500000050011013E0CCC3E9FFCDC3EAFFEECFEA
:1005100000F0AFC3E1FFB0C3E2FF00C0E6FFAF4BA6
:10052000B02BCC4BCD2BC44BC52BE2D7C2A716D0DA
:10053000C0C300F0C1C301F0010EC05F000EC15B7B
:10054000005001100BE0AFC3E1FFB0C3E2FF200E8B
:10055000E66EAF4BB02BC44BC52BEAD793D5B4C3D3
:10056000E9FFB5C3EAFFEECF00F0EECF01F000C027
:10057000E9FF01C0EAFFEECFBFF3B4C3E9FFB5C3A3
:10058000EAFFEECF00F0EECF01F0020E0026000EE3
:100590000122B4C3E1FFB5C3E2FF00C0E6FF01C022
:1005A000E6FFBF0ECC6F030ECD6F010ECE6F000EB7
:1005B000CF6F6AD7C00EC213000EC3133BD0BF511A
:1005C000000AD8B40FD7BF516C0AD8B410D7BF51A6
:1005D000660AD8B40ED7BF51450AD8B40CD7BF515C
:1005E000650AD8B409D7BF51670AD8B407D7BF5135
:1005F0006F0AD8B405D7BF51640AD8B403D7BF5126
:10060000690AD8B4FFD6BF51700AD8B4FCD6BF511E
:10061000580AD8B4F8D6BF51780AD8B4F5D6BF5125
:10062000730AD8B4F3D6BF51630A99E0BF51750A73
:10063000C1E0B7D70301000EC215006EC351070B0E
:10064000016E00500110D8B4A6EF0CF0C3A904D07D
:10065000060EBD6F000EBE6FB4C3E9FFB5C3EAFF5F
:10066000EECF00F0EECF01F000C0E9FF01C0EAFFDD
:10067000EECFC6F3EECFC7F3EECFC8F3EECFC9F39C
:10068000B4C3E9FFB5C3EAFFEECF00F0EECF01F04F
:10069000040E0026000E0122B4C3E1FFB5C3E2FF41
:1006A00000C0E6FF01C0E6FF046A056A066A076A41
:1006B000C6C300F0C7C301F0C8C302F0C9C303F04A
:1006C00022EC30F0010ED8B0000E006E005206E0B1
:1006D0000301C87F030EC213000EC3130301CA6BCC
:1006E000CB6BC6C300F0C7C301F0C8C302F0C9C3D7
:1006F00003F0046A056A066A076A28EC3AF0000EFD
:10070000D8A4010E006E0052D8B49AD0C9C300F02C
:10071000016A026A036AFF0E00140301D46F000E1F
:10072000D56F000ED5177E0ED06F000ED16FD26F31
:10073000D36FD051D45D006ED151D559016E00C038
:10074000CAF301C0CBF3010E005CCA6F000E015862
:10075000CB6FCAC300F0CBC301F0030E046E000ED2
:10076000056E45EC37F000C0CAF301C0CBF30A0EAA
:10077000046E000E056E8AEC30F000C0CAF301C0B2
:10078000CBF3800E01180301D06F800ED05D02E123
:10079000000E005C04E2010ECA5F000ECB5B030199
:1007A000CA510008D86FB3EC18F0C6C304F0C7C331
:1007B00005F0C8C306F0C9C307F017EC2EF000C05F
:1007C000CCF301C0CDF302C0CEF303C0CFF3000ED3
:1007D000046E000E056E000E066E7F0E076ECCC313
:1007E00000F0CDC301F0CEC302F0CFC303F022EC82
:1007F00030F0010ED8B0000E006E005206E0010E7F
:100800000301CA5F000ECB5B1BD0000E046E000E0E
:10081000056E200E066E820E076ECCC300F0CDC3AF
:1008200001F0CEC302F0CFC303F022EC30F0000E93
:10083000D8B0010E006E005203E00301CA4BCB2B6F
:100840000301800E006E800E0301CB19005C02E1F3
:10085000CA51000803E3010EBF6F03D00301CAC3EE
:10086000BFF3C3B11AD0C3A315D0800ECB19006E4D
:100870007F0E005C02E1FC0ECA5D0AE3800ECB191C
:10088000006E800EBE19005C02E1BD51CA5D02E33C
:10089000030103D0030192EF08F00301BD51BE1123
:1008A00006E0C3A304D0010EBD5F000EBE5B000EC8
:1008B000006EBE51005C02E1BD51080803E2080E63
:1008C000BF6F03D00301BDC3BFF3C6C300F0C7C3EE
:1008D00001F0C8C302F0C9C303F0046A056A066ADE
:1008E000076A28EC3AF0000ED8A4010E006E005200
:1008F000D8B464D1CAC3D8F3B3EC18F000C004F084
:1009000001C005F002C006F003C007F0C6C300F046
:10091000C7C301F0C8C302F0C9C303F036EC2CF022
:1009200000C0C6F301C0C7F302C0C8F303C0C9F3D7
:100930000301BF510008D86FB3EC18F000C004F0F9
:1009400001C005F002C006F003C007F0C6C300F006
:10095000C7C301F0C8C302F0C9C303F036EC2CF0E2
:1009600000C0D0F301C0D1F302C0D2F303C0D3F36F
:10097000D0C3C6F3D1C3C7F3D2C3C8F3D3C3C9F33B
:10098000D0C300F0D1C301F0D2C302F0D3C303F04F
:10099000E0EC2CF081EC3AF000C004F001C005F06E
:1009A00002C006F003C007F0D0C300F0D1C301F0CD
:1009B000D2C302F0D3C303F08CEC3BF0000E046E04
:1009C000000E056E000E066E7E0E076E22EC30F0F5
:1009D000000ED8B0010E006E00521AE0C6C300F03F
:1009E000C7C301F0C8C302F0C9C303F0000E046E10
:1009F000000E056E000E066E7E0E076EF2EC1DF008
:100A000000C0C6F301C0C7F302C0C8F303C0C9F3F6
:100A1000C6C300F0C7C301F0C8C302F0C9C303F0E6
:100A2000E0EC2CF000C0D4F301C0D5F302C0D6F343
:100A300003C0D7F30301BF51010F006E016A000E1E
:100A40000122020E046E000E01BEFF0E026E036E46
:100A50000450030107E000360090013602360336E9
:100A6000FF0FF7D70301A20E0026770E0122000E1A
:100A7000022200C0F6FF01C0F7FF02C0F8FF090024
:100A8000F5CFD0F30900F5CFD1F30900F5CFD2F3BC
:100A90000900F5CFD3F3D351D75D08E1D251D65D2C
:100AA00005E1D151D55D02E1D051D45D1EE3C6C34D
:100AB00000F0C7C301F0C8C302F0C9C303F0CD0EF4
:100AC000046ECC0E056E4C0E066E7B0E076E17EC98
:100AD0002EF000C0C6F301C0C7F302C0C8F303C0C4
:100AE000C9F30301CA4BCB2B69D00301C6C300F085
:100AF000C7C301F0C8C302F0C9C303F0E0EC2CF097
:100B000000C0D4F301C0D5F302C0D6F303C0D7F3BD
:100B1000020E046EBFC300F0000E016E026E036E83
:100B20000450000107E0003600900136023603361B
:100B3000FF0FF7D7A20E0026770E0122000E022229
:100B400000C0F6FF01C0F7FF02C0F8FF0900F5CFB3
:100B5000D0F30900F5CFD1F30900F5CFD2F30900A6
:100B6000F5CFD3F30301D351D75D08E1D251D65D60
:100B700005E1D151D55D02E1D051D45D1FE2C6C37C
:100B800000F0C7C301F0C8C302F0C9C303F0000EF0
:100B9000046E000E056E200E066E820E076E17ECB8
:100BA0002EF000C0C6F301C0C7F302C0C8F303C0F3
:100BB000C9F3010E0301CA5F000ECB5B0301030101
:100BC000C3A398D0C3B796D0800E000A006E800EE3
:100BD000BE19005C02E1BD510A0804E20A0EBD6FB5
:100BE000000EBE6F0301C6C300F0C7C301F0C8C347
:100BF00002F0C9C303F0E0EC2CF000C0CCF301C05C
:100C0000CDF302C0CEF303C0CFF30301CC51CD111D
:100C1000CE11CF1144E00A0E046E000E056E066E72
:100C2000076ECCC300F0CDC301F0CEC302F0CFC33A
:100C300003F06FEC23F008C000F009C001F00AC017
:100C400002F00BC003F0000E0301D06F031808E19F
:100C5000D051021805E1D051011802E10050000AFC
:100C60001EE1010E0301BD5F000EBE5B0A0E046EA5
:100C7000000E056E066E076ECCC300F0CDC301F00A
:100C8000CEC302F0CFC303F06FEC23F000C0CCF36F
:100C900001C0CDF302C0CEF303C0CFF3B6D7800EB0
:100CA0000301BE19006E800E005C02E1BF51BD5D04
:100CB00021E2BD51BF5DD86FB3EC18F000C004F065
:100CC00001C005F002C006F003C007F0C6C300F083
:100CD000C7C301F0C8C302F0C9C303F036EC2CF05F
:100CE00000C0C6F301C0C7F302C0C8F303C0C9F314
:100CF000BDC3BFF30001050E0301BD25006E000E4C
:100D0000BE21016E0050C05F0150C15BBD51BE11DC
:100D100002E1C3A704D0010EC05F000EC15B030E49
:100D2000C215006EC3C301F0000E01160050011081
:100D300004E0010EC05F000EC15BC2A54AD0C2A391
:100D40001AD0010EC215006EC3C301F0000E0116C9
:100D50000050011003E02D0E006E02D02B0E006E2D
:100D6000AFC3E1FFB0C3E2FF00C0E6FFAF4BB02B63
:100D7000C44BC52B14D0010EC215006EC3C301F0C5
:100D8000000E0116005001100AE0AFC3E1FFB0C32E
:100D9000E2FF200EE66EAF4BB02BC44BC52B800E8E
:100DA000006E800EC119005C02E1C05100080FE224
:100DB000AFC3E1FFB0C3E2FF300EE66EAF4BB02B26
:100DC000C44BC52B010EC05F000EC15BE8D7030109
:100DD0004BD0C2B718D0800E006E800EC119005CD7
:100DE00002E1C05100080FE2AFC3E1FFB0C3E2FF70
:100DF000200EE66EAF4BB02BC44BC52B010EC05F6F
:100E0000000EC15BE8D70301C2A31AD0010EC215C0
:100E1000006EC3C301F0000E01160050011003E084
:100E20002D0E006E02D02B0E006EAFC3E1FFB0C3DB
:100E3000E2FF00C0E6FFAF4BB02BC44BC52B14D074
:100E4000010EC215006EC3C301F0000E0116005062
:100E500001100AE0AFC3E1FFB0C3E2FF200EE66E6F
:100E6000AF4BB02BC44BC52B0301C6C300F0C7C3A7
:100E700001F0C8C302F0C9C303F0E0EC2CF000C0DD
:100E8000CCF301C0CDF302C0CEF303C0CFF3020E0A
:100E9000046EBFC300F0000E016E026E036E0450BC
:100EA000000107E000360090013602360336FF0FDE
:100EB000F7D7A20E0026770E0122000E022200C0F4
:100EC000F6FF01C0F7FF02C0F8FF0900F5CF04F0FC
:100ED0000900F5CF05F00900F5CF06F00900F5CFC0
:100EE00007F0CCC300F0CDC301F0CEC302F0CFC3F6
:100EF00003F06FEC23F0300E0026AFC3E1FFB0C368
:100F0000E2FF00C0E6FF0301AF4BB02BC44BC52B83
:100F1000BD51BE1102E1C3A776D0AFC3E1FFB0C39C
:100F2000E2FF2E0EE66E0301AF4BB02BC44BC52B78
:100F3000BF51BD5F000EBE5BBF5353E0BF07020E43
:100F4000046EBFC300F0000E016E026E036E04500B
:100F5000030107E000360090013602360336FF0F2A
:100F6000F7D7A20E0026770E0122000E022200C043
:100F7000F6FF01C0F7FF02C0F8FF0900F5CF04F04B
:100F80000900F5CF05F00900F5CF06F00900F5CF0F
:100F900007F0CCC300F0CDC301F0CEC302F0CFC345
:100FA00003F06FEC23F00A0E046E000E056E066E61
:100FB000076E6FEC23F008C000F009C001F00AC012
:100FC00002F00BC003F0300E0026AFC3E1FFB0C348
:100FD000E2FF00C0E6FF0301AF4BB02BC44BC52BB3
:100FE000ABD7BD51BE110FE0AFC3E1FFB0C3E2FF0D
:100FF000300EE66EAF4BB02BC44BC52B010EBD5F60
:10100000000EBE5BEED7C2AB0BD0AFC3E1FFB0C3E7
:10101000E2FF450EE66EAF4BB02BC44BC52B0AD09A
:10102000AFC3E1FFB0C3E2FF650EE66EAF4BB02B7E
:10103000C44BC52B800ECB19006E800E005C02E104
:10104000000ECA5D12E2CA510008CA6FCBC3CBF3CF
:10105000E86ACB57AFC3E1FFB0C3E2FF2D0EE66EE7
:10106000AF4BB02BC44BC52B0BD00301AFC3E1FF7B
:10107000B0C3E2FF2B0EE66EAF4BB02BC44BC52BBB
:101080000A0E046E000E056ECAC300F0CBC301F059
:101090008AEC30F0300E0026AFC3E1FFB0C3E2FFB0
:1010A00000C0E6FF0301AF4BB02BC44BC52B0A0EAB
:1010B000046E000E056ECAC300F0CBC301F08AECCB
:1010C00030F008C000F009C001F0300E0026AFC3B8
:1010D000E1FFB0C3E2FF00C0E6FF0301AF4BB02B5E
:1010E000C44BC52BC2A71BD0800E006E800EC11949
:1010F000005C02E1C051000812E2AFC3E1FFB0C3DF
:10110000E2FF200EE66E0301AF4BB02BC44BC52BA4
:10111000010EC05F000EC15BC051C111EEE10301C1
:1011200042EF00F00301C3A3FDD0800ECB19006E87
:10113000800E005C02E1000ECA5D0AE2010ECA5D8B
:10114000006E000ECB59016E0050BD5F0150BE5BBA
:10115000C6C300F0C7C301F0C8C302F0C9C303F09F
:10116000E0EC2CF000C0CCF301C0CDF302C0CEF314
:1011700003C0CFF3010E0301BF6FBF510A0A39E06C
:10118000020E046EBFC300F0000E016E026E036E0D
:101190000450030107E000360090013602360336A2
:1011A000FF0FF7D70301A20E0026770E0122000ED3
:1011B000022200C0F6FF01C0F7FF02C0F8FF0900DD
:1011C000F5CFD0F30900F5CFD1F30900F5CFD2F375
:1011D0000900F5CFD3F3D351CF5D08E1D251CE5DF5
:1011E00005E1D151CD5D02E1D051CC5D02E3BF2BD1
:1011F000C4D70301BF51BD5DD46F000EBE59D56F7A
:10120000D4C3BDF3D5C3BEF3CCC300F0CDC301F04E
:10121000CEC302F0CFC303F081EC3AF000C004F07B
:1012200001C005F002C006F003C007F0C6C300F01D
:10123000C7C301F0C8C302F0C9C303F08CEC3BF094
:1012400000C0D0F301C0D1F302C0D2F303C0D3F386
:10125000D4C3D8F3B3EC18F0D0C304F0D1C305F075
:10126000D2C306F0D3C307F017EC2EF0000E046EC5
:10127000000E056E000E066E7E0E076EF2EC1DF07F
:10128000E0EC2CF000C0CCF301C0CDF302C0CEF3F3
:1012900003C0CFF30301BD51BE1144E00A0E046E3A
:1012A000000E056E066E076ECCC300F0CDC301F0D4
:1012B000CEC302F0CFC303F06FEC23F008C000F000
:1012C00009C001F00AC002F00BC003F0000E0301D8
:1012D000D06F031808E1D051021805E1D051011870
:1012E00002E10050000A1EE10A0E046E000E056EB7
:1012F000066E076ECCC300F0CDC301F0CEC302F082
:10130000CFC303F06FEC23F000C0CCF301C0CDF3EA
:1013100002C0CEF303C0CFF3010E0301BD5F000E88
:10132000BE5BB8D70301800E006E800E0301BE19AC
:10133000005C02E1BD510C0816E3BDC3D8F3DCEC40
:1013400021F0C6C304F0C7C305F0C8C306F0C9C383
:1013500007F0F2EC1DF000C0C6F301C0C7F302C0F5
:10136000C8F303C0C9F3C6C300F0C7C301F0C8C3C4
:1013700002F0C9C303F0046A056A066A076A28EC2A
:101380003AF0000ED8A4010E006E0052D8B478D006
:10139000C6C300F0C7C301F0C8C302F0C9C303F05D
:1013A000E0EC2CF0000E0301D06F031808E1D051DF
:1013B000021805E1D051011802E10050000A60E175
:1013C000800E006E800ECB19005C02E1CA5101084C
:1013D00057E2CAC3D8F3B3EC18F000C004F001C060
:1013E00005F002C006F003C007F0C6C300F0C7C393
:1013F00001F0C8C302F0C9C303F036EC2CF05F0E55
:10140000046E700E056E090E066E810E076E22ECDC
:1014100030F0010ED8B0000E006E005206E0090E4A
:101420000301CA5F000ECB5B05D0080E0301CA5F43
:10143000000ECB5BCAC3D8F3B3EC18F000C004F0C5
:1014400001C005F002C006F003C007F0C6C300F0FB
:10145000C7C301F0C8C302F0C9C303F036EC2CF0D7
:10146000E0EC2CF000C0CCF301C0CDF302C0CEF311
:1014700003C0CFF30301C66BC76BC86BC96B39D010
:10148000C6C300F0C7C301F0C8C302F0C9C303F06C
:10149000E0EC2CF000C0CCF301C0CDF302C0CEF3E1
:1014A00003C0CFF3CCC300F0CDC301F0CEC302F034
:1014B000CFC303F081EC3AF000C004F001C005F0A6
:1014C00002C006F003C007F0C6C300F0C7C301F0B6
:1014D000C8C302F0C9C303F08CEC3BF000C0C6F3F4
:1014E00001C0C7F302C0C8F303C0C9F30301CA6B4C
:1014F000CB6B010EBF6FBF510A0A39E0020E046EBA
:10150000BFC300F0000E016E026E036E04500301B3
:1015100007E000360090013602360336FF0FF7D79A
:101520000301A20E0026770E0122000E022200C047
:10153000F6FF01C0F7FF02C0F8FF0900F5CFD0F3B6
:101540000900F5CFD1F30900F5CFD2F30900F5CFAB
:10155000D3F3D351CF5D08E1D251CE5D05E1D15136
:10156000CD5D02E1D051CC5D02E3BF2BC4D70301B6
:10157000BF51BD25006E000EBE21016ECA5100266E
:10158000CB5101220050C05F0150C15BC3B703D0F3
:10159000BD51BE1104E0010EC05F000EC15B030E21
:1015A000C215006EC3C301F0000E011600500110F9
:1015B00004E0010EC05F000EC15BC2A54AD0C2A309
:1015C0001AD0010EC215006EC3C301F0000E011641
:1015D0000050011003E02D0E006E02D02B0E006EA5
:1015E000AFC3E1FFB0C3E2FF00C0E6FFAF4BB02BDB
:1015F000C44BC52B14D0010EC215006EC3C301F03D
:10160000000E0116005001100AE0AFC3E1FFB0C3A5
:10161000E2FF200EE66EAF4BB02BC44BC52B800E05
:10162000006E800EC119005C02E1C05100080FE29B
:10163000AFC3E1FFB0C3E2FF300EE66EAF4BB02B9D
:10164000C44BC52B010EC05F000EC15BE8D7030180
:101650004BD0C2B718D0800E006E800EC119005C4E
:1016600002E1C05100080FE2AFC3E1FFB0C3E2FFE7
:10167000200EE66EAF4BB02BC44BC52B010EC05FE6
:10168000000EC15BE8D70301C2A31AD0010EC21538
:10169000006EC3C301F0000E01160050011003E0FC
:1016A0002D0E006E02D02B0E006EAFC3E1FFB0C353
:1016B000E2FF00C0E6FFAF4BB02BC44BC52B14D0EC
:1016C000010EC215006EC3C301F0000E01160050DA
:1016D00001100AE0AFC3E1FFB0C3E2FF200EE66EE7
:1016E000AF4BB02BC44BC52B0301BFC300F0BF07EA
:1016F000005252E0020E046EBFC300F0000E016EF5
:10170000026E036E0450030107E0003600900136BC
:1017100002360336FF0FF7D7A20E0026770E0122FE
:10172000000E022200C0F6FF01C0F7FF02C0F8FF62
:101730000900F5CF04F00900F5CF05F00900F5CF59
:1017400006F00900F5CF07F0CCC300F0CDC301F0DF
:10175000CEC302F0CFC303F06FEC23F00A0E046E89
:10176000000E056E066E076E6FEC23F008C000F0E9
:1017700009C001F00AC002F00BC003F0300E0026D1
:10178000AFC3E1FFB0C3E2FF00C0E6FF0301AF4B10
:10179000B02BC44BC52BA8D7800E006E800ECB1982
:1017A000005C02E1CA5100080FE2AFC3E1FFB0C321
:1017B000E2FF300EE66EAF4BB02BC44BC52B010ED3
:1017C000CA5F000ECB5BE8D70301800E000A006EF3
:1017D000800EBE19005C02E1BD51080803E2080E4C
:1017E000BF6F03D00301BDC3BFF3BF51BD5F000E88
:1017F000BE5BBF5302E1C3A70AD0AFC3E1FFB0C3D2
:10180000E2FF2E0EE66EAF4BB02BC44BC52BBFC311
:10181000D8F3B3EC18F0C6C304F0C7C305F0C8C3CF
:1018200006F0C9C307F017EC2EF07DEC2DF000C0D8
:10183000CCF301C0CDF302C0CEF303C0CFF303015C
:10184000BF5353E0BF07020E046EBFC300F0000E8B
:10185000016E026E036E0450030107E00036009033
:10186000013602360336FF0FF7D7A20E0026770E99
:101870000122000E022200C0F6FF01C0F7FF02C0E5
:10188000F8FF0900F5CF04F00900F5CF05F00900D5
:10189000F5CF06F00900F5CF07F0CCC300F0CDC3BB
:1018A00001F0CEC302F0CFC303F06FEC23F00A0EB9
:1018B000046E000E056E066E076E6FEC23F008C016
:1018C00000F009C001F00AC002F00BC003F0300EB6
:1018D0000026AFC3E1FFB0C3E2FF00C0E6FF030193
:1018E000AF4BB02BC44BC52BAAD7BD51BE110FE0D7
:1018F000AFC3E1FFB0C3E2FF300EE66EAF4BB02BDB
:10190000C44BC52B010EBD5F000EBE5BEED7C2A758
:101910001AD0800E006E800EC119005C02E1C05129
:10192000000811E2AFC3E1FFB0C3E2FF200EE66E94
:10193000AF4BB02BC44BC52B010EC05F000EC15B7B
:10194000C051C111EFE1030142EF00F0C00EC2151A
:10195000D06FC3C3D1F3000ED117000ED11902E12D
:10196000000ED019D8A482D0C2A929D0B4C3E9FFEF
:10197000B5C3EAFFEECF00F0EECF01F000C0E9FF03
:1019800001C0EAFFEECFCCF3EECFCDF3EECFCEF336
:10199000EECFCFF3B4C3E9FFB5C3EAFFEECF00F05B
:1019A000EECF01F0040E0026000E0122B4C3E1FFC9
:1019B000B5C3E2FF00C0E6FF01C0E6FF2ED0B4C30E
:1019C000E9FFB5C3EAFFEECF00F0EECF01F000C0B3
:1019D000E9FF01C0EAFFEECFCCF3EECFCDF3000E6E
:1019E000CDBFFF0ECE6FCF6F000ECDBFFF0ECE6FFF
:1019F000CF6FB4C3E9FFB5C3EAFFEECF00F0EECF7F
:101A000001F0020E0026000E0122B4C3E1FFB5C3AF
:101A1000E2FF00C0E6FF01C0E6FF800ECF19006EB6
:101A2000800E005C08E1000ECE5D05E1000ECD5D8C
:101A300002E1000ECC5D18E2030EC213000EC313C8
:101A4000006A016A026A036ACC51005ECD51015AF4
:101A5000CE51025ACF51035A00C0CCF301C0CDF38E
:101A600002C0CEF303C0CFF3030156D00301C2A9D5
:101A700029D0B4C3E9FFB5C3EAFFEECF00F0EECF43
:101A800001F000C0E9FF01C0EAFFEECFCCF3EECFDA
:101A9000CDF3EECFCEF3EECFCFF3B4C3E9FFB5C3B2
:101AA000EAFFEECF00F0EECF01F0040E0026000EAC
:101AB0000122B4C3E1FFB5C3E2FF00C0E6FF01C0ED
:101AC000E6FF2AD0B4C3E9FFB5C3EAFFEECF00F0CA
:101AD000EECF01F000C0E9FF01C0EAFFEECFCCF38A
:101AE000EECFCDF3000ECE6FCF6F000ECE6FCF6F67
:101AF000B4C3E9FFB5C3EAFFEECF00F0EECF01F0CB
:101B0000020E0026000E0122B4C3E1FFB5C3E2FFBE
:101B100000C0E6FF01C0E6FF0301000EBE1902E1AE
:101B2000000EBD190FE1000E006ECF1908E1005044
:101B3000CE1905E10050CD1902E1CC51000A02E1B5
:101B4000BD4BBE2B0301C00EC215006E00C0D4F306
:101B5000C0D0010EBF6FBF510A0A39E0020E046EF9
:101B6000BFC300F0000E016E026E036E045003014D
:101B700007E000360090013602360336FF0FF7D734
:101B80000301A20E0026770E0122000E022200C0E1
:101B9000F6FF01C0F7FF02C0F8FF0900F5CFD0F350
:101BA0000900F5CFD1F30900F5CFD2F30900F5CF45
:101BB000D3F3D351CF5D08E1D251CE5D05E1D151D0
:101BC000CD5D02E1D051CC5D02E3BF2BC4D7030150
:101BD0008FD0010EBF6FBF51080A39E0020E046EAC
:101BE000BFC300F0000E016E026E036E04500301CD
:101BF00007E000360090013602360336FF0FF7D7B4
:101C00000301CA0E0026770E0122000E022200C038
:101C1000F6FF01C0F7FF02C0F8FF0900F5CFD0F3CF
:101C20000900F5CFD1F30900F5CFD2F30900F5CFC4
:101C3000D3F3D351CF5D08E1D251CE5D05E1D1514F
:101C4000CD5D02E1D051CC5D02E3BF2BC4D70301CF
:101C50004FD0010EBF6FBF510C0A39E0020E046E67
:101C6000BFC300F0000E016E026E036E045003014C
:101C700007E000360090013602360336FF0FF7D733
:101C80000301EA0E0026770E0122000E022200C098
:101C9000F6FF01C0F7FF02C0F8FF0900F5CFD0F34F
:101CA0000900F5CFD1F30900F5CFD2F30900F5CF44
:101CB000D3F3D351CF5D08E1D251CE5D05E1D151CF
:101CC000CD5D02E1D051CC5D02E3BF2BC4D703014F
:101CD0000FD0D451000AD8B43CD7D451C00AD8B4DC
:101CE00038D7D451800AD8B474D7D451400AB1E05F
:101CF0000301800E006E800EBE19005C02E1BD5132
:101D0000BF5D03E2BDC3BFF30ED00301800EBE1959
:101D1000006E800E005C02E1BF51BD5D04E2BFC3F6
:101D2000BDF3000EBE6F03010301C051C1110EE0EF
:101D3000030EC215006EC3C301F0000E0116005061
:101D4000011004E0010EC05F000EC15B800EBE19E1
:101D5000006E800EC119005C02E1C051BD5D05E25C
:101D6000BD51C05FBE51C15B03D00301C06BC16BED
:101D7000C40EC215D06FC351080BD16FD151080AE0
:101D800002E1400ED01908E1C051C11104E0010E7A
:101D9000C05F000EC15B1ED00301C00EC215D06F24
:101DA000C351080BD16FD151080A02E1800ED0193E
:101DB00011E1800E006E800EC119005C02E1C0517D
:101DC000020805E2020EC05F000EC15B03D00301F2
:101DD000C06BC16B03010301C2A56ED0C2A31AD0B0
:101DE000010EC215006EC3C301F0000E01160050B3
:101DF000011003E02D0E006E02D02B0E006EAFC35B
:101E0000E1FFB0C3E2FF00C0E6FFAF4BB02BC44B15
:101E1000C52B3CD0010EC215006EC3C301F0000EED
:101E20000116005001100BE0AFC3E1FFB0C3E2FFA9
:101E3000200EE66EAF4BB02BC44BC52B27D0C00E87
:101E4000C215D06FC351080BD16FD151080A02E1FE
:101E5000800ED0191BE1AFC3E1FFB0C3E2FF300E2B
:101E6000E66EAF4BB02BC44BC52BC2AB03D0580EA4
:101E7000006E02D0780E006EAFC3E1FFB0C3E2FF88
:101E800000C0E6FFAF4BB02BC44BC52B0301C051C4
:101E9000C11111E0AFC3E1FFB0C3E2FF300EE66E47
:101EA000AF4BB02BC44BC52B010EC05F000EC15B06
:101EB000C051C111EFE185D0C051C11113E0C2B7CB
:101EC00011D0AFC3E1FFB0C3E2FF200EE66EAF4B0F
:101ED000B02BC44BC52B010EC05F000EC15BC051BF
:101EE000C111EFE1C2A31AD0010EC215006EC3C327
:101EF00001F0000E01160050011003E02D0E006EDF
:101F000002D02B0E006EAFC3E1FFB0C3E2FF00C0F2
:101F1000E6FFAF4BB02BC44BC52B14D0010EC2153E
:101F2000006EC3C301F0000E0116005001100AE05C
:101F3000AFC3E1FFB0C3E2FF200EE66EAF4BB02BA4
:101F4000C44BC52BC00EC215D06FC351080BD16F47
:101F5000D151080A02E1400ED0190BE1AFC3E1FFF5
:101F6000B0C3E2FF300EE66EAF4BB02BC44BC52BB7
:101F700028D00301C00EC215D06FC351080BD16F1A
:101F8000D151080A02E1800ED0191BE1AFC3E1FF75
:101F9000B0C3E2FF300EE66EAF4BB02BC44BC52B87
:101FA000C2AB03D0580E006E02D0780E006EAFC3E5
:101FB000E1FFB0C3E2FF00C0E6FFAF4BB02BC44B64
:101FC000C52B03010301800E006E800EBE19005C5C
:101FD00002E1BD51BF5D0BE2AFC3E1FFB0C3E2FF61
:101FE000300EE66EAF4BB02BC44BC52BEAD70301C6
:101FF000BDC300F0BEC301F0010EBD5F000EBE5BAD
:1020000000500110D8B44DD1C00EC215006E00C0F2
:10201000D0F32BD1020E046EBDC300F0BEC301F09D
:10202000000EBEBFFF0E026E036E0450030107E0F8
:1020300000360090013602360336FF0FF7D7A20EA6
:102040000026770E0122000E022200C0F6FF01C01A
:10205000F7FF02C0F8FF0900F5CF04F00900F5CF43
:1020600005F00900F5CF06F00900F5CF07F0CCC365
:1020700000F0CDC301F0CEC302F0CFC303F06FEC8C
:1020800023F00A0E046E000E056E066E076E6FECEE
:1020900023F008C000F009C001F00AC002F00BC034
:1020A00003F0300E00240301BF6FEFD0C2AB4ED05F
:1020B000020E046EBDC300F0BEC301F0000EBEBF31
:1020C000FF0E026E036E0450030107E0003600901D
:1020D000013602360336FF0FF7D70301CA0E00267A
:1020E000770E0122000E022200C0F6FF01C0F7FFAA
:1020F00002C0F8FF0900F5CF04F00900F5CF05F0A4
:102100000900F5CF06F00900F5CF07F0CCC300F0C9
:10211000CDC301F0CEC302F0CFC303F06FEC23F0C8
:102120000F0E0016000E0116021603161A0E0026D8
:10213000780E0122000E022200C0F6FF01C0F7FF58
:1021400002C0F8FF0900F5CFBFF34ED0020E046EB7
:10215000BDC300F0BEC301F0000E0301BEBFFF0E01
:10216000026E036E0450030107E000360090013652
:1021700002360336FF0FF7D70301CA0E0026770E8B
:102180000122000E022200C0F6FF01C0F7FF02C0CC
:10219000F8FF0900F5CF04F00900F5CF05F00900BC
:1021A000F5CF06F00900F5CF07F0CCC300F0CDC3A2
:1021B00001F0CEC302F0CFC303F06FEC23F00F0E9B
:1021C0000016000E0116021603162C0E0026780EBD
:1021D0000122000E022200C0F6FF01C0F7FF02C07C
:1021E000F8FF0900F5CFBFF300014FD0020E046ED7
:1021F000BDC300F0BEC301F0000E0301BEBFFF0E61
:10220000026E036E0450030107E0003600900136B1
:1022100002360336FF0FF7D7EA0E0026770E0122AB
:10222000000E022200C0F6FF01C0F7FF02C0F8FF57
:102230000900F5CF04F00900F5CF05F00900F5CF4E
:1022400006F00900F5CF07F0CCC300F0CDC301F0D4
:10225000CEC302F0CFC303F06FEC23F0070E0014DF
:102260000301BF6F300EBF2710D00301D051000A09
:10227000D8B4D0D6D051C00AD8B4CCD6D051800A68
:10228000D8B414D7D051400AB1E00301AFC3E1FF85
:10229000B0C3E2FFBFC3E6FFAF4BB02BC44BC52BAF
:1022A000A6D6C2A71AD0800E006E800EC119005C9F
:1022B00002E1C051000811E2AFC3E1FFB0C3E2FF89
:1022C000200EE66EAF4BB02BC44BC52B010EC05F8A
:1022D000000EC15BC051C111EFE1030142EF00F0FC
:1022E000C4C300F0C5C301F012006E0E0301776F86
:1022F0006F0E786F6E0E796F2D0E7A6F6C0E7B6F8E
:102300006F0E7C6F6E0E7D6F670E7E6F200E7F6F7F
:10231000700E806F720E816F690E826F6E0E836F0A
:10232000740E846F660E856F866B6E0E876F6F0EF0
:10233000886F6E0E896F2D0E8A6F660E8B6F6C0E16
:102340008C6F6F0E8D6F610E8E6F740E8F6F200EFF
:10235000906F700E916F720E926F690E936F6E0E8A
:10236000946F740E956F660E966F976B280E986F2C
:102370006E0E996F750E9A6F6C0E9B6F6C0E9C6F44
:10238000290E9D6F9E6BA66BA76BA46BA56B0301BB
:1023900072C300F073C301F074C302F0010E722720
:1023A000000E7323742300C0F6FF01C0F7FF02C0C4
:1023B000F8FF0900F5CF00F000C0A1F30052D8B437
:1023C000AEEF18F0A151250A0BE070C3E1FF71C315
:1023D000E2FFA1C3E6FF704B712BA64BA72BD7D70B
:1023E000A26BA36BA46BA56B030123D0A487010E82
:1023F0007227000E732374235AD0A481010E722712
:10240000000E7323742353D0A483010E7227000E91
:10241000732374234CD0A587010E7227000E7323FB
:10242000742345D0A485010E7227000E73237423F4
:102430003ED0030172C3F6FF73C3F7FF74C3F8FF06
:102440000900F5CFACF3AC512D0AD0E072C3F6FF12
:1024500073C3F7FF74C3F8FF0900F5CFACF3AC51B9
:10246000200ACBE072C3F6FF73C3F7FF74C3F8FF13
:102470000900F5CFACF3AC512B0AC6E072C3F6FFEE
:1024800073C3F7FF74C3F8FF0900F5CFACF3AC5189
:10249000230AC1E072C3F6FF73C3F7FF74C3F8FFEA
:1024A0000900F5CFACF3AC51300ABCE001D09CD7A9
:1024B0000301A4B3A491A4B7A49572C3F6FF73C398
:1024C000F7FF74C3F8FF0900F5CF00F0000E016EAE
:1024D00000C0D8F337EC3BF0005238E00301A26BA8
:1024E000A36BA2C300F0A3C301F00A0E046E000E9A
:1024F000056E45EC37F072C3F6FF73C3F7FF74C384
:10250000F8FF0900F5CFACF30301AC510024A26F32
:10251000000E0120A36F300EA25F000EA35B010E20
:102520007227000E7323742372C3F6FF73C3F7FF81
:1025300074C3F8FF0900F5CF00F0000E016E00C073
:10254000D8F337EC3BF00052CCE136D072C3F6FF43
:1025500073C3F7FF74C3F8FF0900F5CFACF30301B1
:10256000AC512A0A29E175C3E9FF76C3EAFFEECF31
:1025700000F0EECF01F000C0E9FF01C0EAFFEECFAE
:10258000A2F3EECFA3F375C3E9FF76C3EAFFEECF64
:1025900000F0EECF01F0020E0026000E012275C3FE
:1025A000E1FF76C3E2FF00C0E6FF01C0E6FF010ED7
:1025B0007227000E73237423030172C3F6FF73C3E3
:1025C000F7FF74C3F8FF0900F5CFACF3AC512E0A46
:1025D00074E1010E7227000E7323742372C3F6FF99
:1025E00073C3F7FF74C3F8FF0900F5CFACF3AC5128
:1025F0002A0A2AE175C3E9FF76C3EAFFEECF00F0AD
:10260000EECF01F000C0E9FF01C0EAFFEECF9FF37B
:10261000EECFA0F375C3E9FF76C3EAFFEECF00F07B
:10262000EECF01F0020E0026000E012275C3E1FF7D
:1026300076C3E2FF00C0E6FF01C0E6FF010E72278D
:10264000000E7323742337D09F6BA06B72C3F6FF09
:1026500073C3F7FF74C3F8FF0900F5CF00F0000E55
:10266000016E00C0D8F337EC3BF0005224E09FC36A
:1026700000F0A0C301F00A0E046E000E056E45ECDA
:1026800037F072C3F6FF73C3F7FF74C3F8FF090096
:10269000F5CFACF30301AC5100249F6F000E012075
:1026A000A06F300E9F5F000EA05B010E7227000E20
:1026B00073237423CBD7030103D003019F6BA06B5B
:1026C000030172C300F073C301F074C302F0010E82
:1026D0007227000E7323742300C0F6FF01C0F7FFBA
:1026E00002C0F8FF0900F5CFA1F302D1A6C300F0A4
:1026F000A7C301F01200770EA86F030EA96F9F6B9E
:10270000A06BFF0EA46FFF0EA56F31D0870EA86FD0
:10271000030EA96F9F6BA06B2AD0A48D24D123D167
:10272000A48BA48F20D175C3E9FF76C3EAFFEECF57
:1027300000F0EECF01F000C0E9FF01C0EAFFEECFEC
:10274000A8F3EECFA9F375C3E9FF76C3EAFFEECF96
:1027500000F0EECF01F0020E0026000E012275C33C
:10276000E1FF76C3E2FF00C0E6FF01C0E6FF000E16
:10277000A91902E1000EA81904E1980EA86F030E32
:10278000A96F0301AA6BAB6BAA51A825E96EAB51E7
:10279000A921EA6EEECF00F0005203E0AA4BAB2B6A
:1027A000F3D79F51A0110AE0AB51A05D02E1AA51FD
:1027B0009F5D04E29FC3AAF3A0C3ABF30301A3513F
:1027C000AB5D02E1A251AA5D05E2AA51A25FAB5145
:1027D000A35B03D00301A26BA36BA4B716D0A2C363
:1027E00000F0A3C301F0010EA25F000EA35B005036
:1027F00001100BE070C3E1FF71C3E2FF200EE66E33
:10280000704B712BA64BA72BEAD7AAC300F0ABC322
:1028100001F0010EAA5F000EAB5B0050011013E047
:10282000A8C3E9FFA9C3EAFFEECF00F070C3E1FF40
:1028300071C3E2FF00C0E6FF704B712BA84BA92BC0
:10284000A64BA72BE2D7A4A716D0A2C300F0A3C320
:1028500001F0010EA25F000EA35B005001100BE01F
:1028600070C3E1FF71C3E2FF200EE66E704B712B67
:10287000A64BA72BEAD7A551FF0A02E1FF0EA41928
:1028800005E1A6C300F0A7C301F0120003017FD544
:1028900075C3E9FF76C3EAFFEECF00F0EECF01F09B
:1028A00000C0E9FF01C0EAFFEECFA1F375C3E9FF65
:1028B00076C3EAFFEECF00F0EECF01F0020E002665
:1028C000000E012275C3E1FF76C3E2FF00C0E6FF00
:1028D00001C0E6FFA10EA86F030EA96F010EAA6F3B
:1028E000000EAB6F5ED7C00EA413000EA5133BD035
:1028F000A151000AD8B4FAD6A1516C0AD8B4FBD6BB
:10290000A151450AD8B402D7A151660AD8B4FED65F
:10291000A151650AD8B4FAD6A151670AD8B4F6D63F
:10292000A1516F0AD8B4F9D6A151640AD8B4F7D628
:10293000A151690AD8B4F3D6A151700AD8B4F0D61F
:10294000A151580AD8B4ECD6A151780AD8B4E9D626
:10295000A151730AD8B4E7D6A151630A99E0A151F5
:10296000750AC1E0B7D70301C00EA415AC6FA5C3AB
:10297000ADF3000EAD17000EAD1902E1000EAC195B
:102980003EE175C3E9FF76C3EAFFEECF00F0EECF7C
:1029900001F000C0E9FF01C0EAFFEECFA8F3EECFDF
:1029A000A9F375C3E9FF76C3EAFFEECF00F0EECFDF
:1029B00001F0020E0026000E012275C3E1FF76C36E
:1029C000E2FF00C0E6FF01C0E6FF800EA919006E1D
:1029D000800E005C02E1000EA85D0FE2030EA4135E
:1029E000000EA513A8510008006EA9C301F0E86A03
:1029F000015600C0A8F301C0A9F3030125D00301CB
:102A000075C3E9FF76C3EAFFEECF00F0EECF01F029
:102A100000C0E9FF01C0EAFFEECFA8F3EECFA9F3B3
:102A200075C3E9FF76C3EAFFEECF00F0EECF01F009
:102A3000020E0026000E012275C3E1FF76C3E2FFFD
:102A400000C0E6FF01C0E6FF0301000EA01902E18D
:102A5000000E9F1908E1000EA91902E1000EA81945
:102A600002E19F4BA02B0301C00EA415006E00C015
:102A7000AEF39CD0010EA16FA151050A2DE0010E0D
:102A8000046EA1C300F0000E016E026E036E0450CE
:102A9000030107E000360090013602360336FF0FCF
:102AA000F7D703013E0E0026780E0122000E022207
:102AB00000C0F6FF01C0F7FF02C0F8FF0900F5CF24
:102AC000ACF30900F5CFADF3AD51A95D02E1AC5116
:102AD000A85D02E3A12BD0D7030176D0010EA16F30
:102AE000A151040A2DE0010E046EA1C300F0000EF6
:102AF000016E026E036E0450030107E00036009081
:102B0000013602360336FF0FF7D70301480E0026C1
:102B1000780E0122000E022200C0F6FF01C0F7FF6E
:102B200002C0F8FF0900F5CFACF30900F5CFADF313
:102B3000AD51A95D02E1AC51A85D02E3A12BD0D754
:102B4000030142D0010EA16FA151060A2DE0010E32
:102B5000046EA1C300F0000E016E026E036E0450FD
:102B6000030107E000360090013602360336FF0FFE
:102B7000F7D70301500E0026780E0122000E022224
:102B800000C0F6FF01C0F7FF02C0F8FF0900F5CF53
:102B9000ACF30900F5CFADF3AD51A95D02E1AC5145
:102BA000A85D02E3A12BD0D703010ED0AE51000ADD
:102BB000D8B460D7AE51C00AD8B45CD7AE51800A41
:102BC0008DE0AE51400ABEE00301800E006E800E23
:102BD000A019005C02E19F51A15D03E29FC3A1F334
:102BE0000ED00301800EA019006E800E005C02E181
:102BF000A1519F5D04E2A1C39FF3000EA06F0301EA
:102C00000301A251A3110EE0030EA415006EA5C38B
:102C100001F0000E01160050011004E0010EA25F49
:102C2000000EA35B800EA019006E800EA319005C3D
:102C300002E1A2519F5D05E29F51A25FA051A35BFB
:102C400003D00301A26BA36BC40EA415AC6FA551F6
:102C5000080BAD6FAD51080A02E1400EAC1908E156
:102C6000A251A31104E0010EA25F000EA35B1ED0CF
:102C70000301C00EA415AC6FA551080BAD6FAD518B
:102C8000080A02E1800EAC1911E1800E006E800E80
:102C9000A319005C02E1A251020805E2020EA25F44
:102CA000000EA35B03D00301A26BA36B030103011E
:102CB000A4A56ED0A4A31AD0010EA415006EA5C3BE
:102CC00001F0000E01160050011003E02D0E006E01
:102CD00002D02B0E006E70C3E1FF71C3E2FF00C093
:102CE000E6FF704B712BA64BA72B3CD0010EA41511
:102CF000006EA5C301F0000E0116005001100BE09C
:102D000070C3E1FF71C3E2FF200EE66E704B712BC2
:102D1000A64BA72B27D0C00EA415AC6FA551080B4E
:102D2000AD6FAD51080A02E1800EAC191BE170C312
:102D3000E1FF71C3E2FF300EE66E704B712BA64BC4
:102D4000A72BA4AB03D0580E006E02D0780E006EF5
:102D500070C3E1FF71C3E2FF00C0E6FF704B712B4F
:102D6000A64BA72B0301A251A31111E070C3E1FFF1
:102D700071C3E2FF300EE66E704B712BA64BA72B92
:102D8000010EA25F000EA35BA251A311EFE185D05B
:102D9000A251A31113E0A4B711D070C3E1FF71C316
:102DA000E2FF200EE66E704B712BA64BA72B010E97
:102DB000A25F000EA35BA251A311EFE1A4A31AD05E
:102DC000010EA415006EA5C301F0000E01160050FF
:102DD000011003E02D0E006E02D02B0E006E70C3AA
:102DE000E1FF71C3E2FF00C0E6FF704B712BA64B01
:102DF000A72B14D0010EA415006EA5C301F0000E80
:102E00000116005001100AE070C3E1FF71C3E2FF38
:102E1000200EE66E704B712BA64BA72BC00EA4158F
:102E2000AC6FA551080BAD6FAD51080A02E1400E21
:102E3000AC190BE170C3E1FF71C3E2FF300EE66E27
:102E4000704B712BA64BA72B28D00301C00EA415E5
:102E5000AC6FA551080BAD6FAD51080A02E1800EB1
:102E6000AC191BE170C3E1FF71C3E2FF300EE66EE7
:102E7000704B712BA64BA72BA4AB03D0580E006E42
:102E800002D0780E006E70C3E1FF71C3E2FF00C094
:102E9000E6FF704B712BA64BA72B03010301800E9D
:102EA000006E800EA019005C02E19F51A15D0BE253
:102EB00070C3E1FF71C3E2FF300EE66E704B712B01
:102EC000A64BA72BEAD703019FC300F0A0C301F0D4
:102ED000010E9F5F000EA05B00500110D8B41FD1FF
:102EE000C00EA415006E00C0ACF3FDD0010E046E40
:102EF0009FC300F0A0C301F0000EA0BFFF0E026E42
:102F0000036E0450030107E00036009001360236DC
:102F10000336FF0FF7D73E0E0026780E0122000E73
:102F2000022200C0F6FF01C0F7FF02C0F8FF09004F
:102F3000F5CF04F00900F5CF05F0A8C300F0A9C350
:102F400001F09EEC39F00A0E046E000E056E9EEC48
:102F500039F008C000F009C001F0300E0024030170
:102F6000A16FD1D0A4AB44D0010E046E9FC300F07A
:102F7000A0C301F0000EA0BFFF0E026E036E04504E
:102F8000030107E000360090013602360336FF0FDA
:102F9000F7D70301480E0026780E0122000E022208
:102FA00000C0F6FF01C0F7FF02C0F8FF0900F5CF2F
:102FB00004F00900F5CF05F0A8C300F0A9C301F0A3
:102FC0009EEC39F00F0E0016000E0116000E026E78
:102FD0005C0E0026780E0122000E022200C0F6FFD1
:102FE00001C0F7FF02C0F8FF0900F5CFA1F344D0FC
:102FF000010E046E9FC300F0A0C301F0000E030198
:10300000A0BFFF0E026E036E0450030107E00036FE
:103010000090013602360336FF0FF7D70301480E42
:103020000026780E0122000E022200C0F6FF01C029
:10303000F7FF02C0F8FF0900F5CF04F00900F5CF53
:1030400005F0A8C300F0A9C301F09EEC39F00F0E03
:103050000016000E0116000E026E6E0E0026780E8F
:103060000122000E022200C0F6FF01C0F7FF02C0DD
:10307000F8FF0900F5CFA1F3000145D0010E046E61
:103080009FC300F0A0C301F0000E0301A0BFFF0E1C
:10309000026E036E0450030107E000360090013613
:1030A00002360336FF0FF7D7500E0026780E0122A6
:1030B000000E022200C0F6FF01C0F7FF02C0F8FFB9
:1030C0000900F5CF04F00900F5CF05F0A8C300F022
:1030D000A9C301F09EEC39F0070E00140301A16FA3
:1030E000300EA12710D00301AC51000AD8B4FED68F
:1030F000AC51C00AD8B4FAD6AC51800AD8B432D791
:10310000AC51400ABBE0030170C3E1FF71C3E2FFB1
:10311000A1C3E6FF704B712BA64BA72BD4D6A4A757
:103120001AD0800E006E800EA319005C02E1A2513D
:10313000000811E270C3E1FF71C3E2FF200EE66EEA
:10314000704B712BA64BA72B010EA25F000EA35B49
:10315000A251A311EFE10301C7EF11F0A6C300F0E4
:10316000A7C301F01200800E0301D819006E800E73
:10317000000A005CD8B081D1D8510008046E04C0A8
:10318000D8F3800E0418006E800E6E0A005CD8A082
:10319000C6D0640E046ED8C300F078EC32F0120E84
:1031A0000026000E00BEFF0E016E000E0122020E70
:1031B000046E000E01BEFF0E026E036E045000018D
:1031C00007E000360090013602360336FF0FF7D7CE
:1031D00000013A0E0026770E0122000E022200C0E6
:1031E000F6FF01C0F7FF02C0F8FF0900F5CFD9F3E1
:1031F0000900F5CFDAF30900F5CFDBF30900F5CFCD
:10320000DCF3640E046ED8C300F078EC32F008C032
:1032100000F00A0E046E78EC32F0090E0026000E63
:1032200000BEFF0E016E000E0122020E046E000EA3
:1032300001BEFF0E026E036E0450000107E000366F
:103240000090013602360336FF0FF7D700013A0E21
:103250000026770E0122000E022200C0F6FF01C0F8
:10326000F7FF02C0F8FF0900F5CF00F00900F5CF25
:1032700001F00900F5CF02F00900F5CF03F0D9C342
:1032800004F0DAC305F0DBC306F0DCC307F017EC8B
:103290002EF000C0D9F301C0DAF302C0DBF303C0A3
:1032A000DCF30A0E046ED8C300F078EC32F008C0EC
:1032B00000F0020E046E000E00BEFF0E016E026EE4
:1032C000036E0450000107E000360090013602361C
:1032D0000336FF0FF7D700013A0E0026770E0122C2
:1032E000000E022200C0F6FF01C0F7FF02C0F8FF87
:1032F0000900F5CF00F00900F5CF01F00900F5CF86
:1033000002F00900F5CF03F0D9C304F0DAC305F0E9
:10331000DBC306F0DCC307F017EC2EF01200800EC2
:103320000A0A006E800E0301D819005C76E20A0ECC
:10333000046ED8C300F078EC32F0090E0026000EBF
:1033400000BEFF0E016E000E0122020E046E000E82
:1033500001BEFF0E026E036E0450000107E000364E
:103360000090013602360336FF0FF7D700013A0E00
:103370000026770E0122000E022200C0F6FF01C0D7
:10338000F7FF02C0F8FF0900F5CFD9F30900F5CF28
:10339000DAF30900F5CFDBF30900F5CFDCF30A0E11
:1033A000046ED8C300F078EC32F008C000F0020ED2
:1033B000046E000E00BEFF0E016E026E036E04501E
:1033C000000107E000360090013602360336FF0F99
:1033D000F7D700013A0E0026770E0122000E0222D6
:1033E00000C0F6FF01C0F7FF02C0F8FF0900F5CFEB
:1033F00000F00900F5CF01F00900F5CF02F0090057
:10340000F5CF03F0D9C304F0DAC305F0DBC306F04F
:10341000DCC307F017EC2EF012000001020E046E60
:10342000D8C300F0000E0301D8BFFF0E016E026E7C
:10343000036E0450030107E00036009001360236A7
:103440000336FF0FF7D703013A0E0026770E01224D
:10345000000E022200C0F6FF01C0F7FF02C0F8FF15
:103460000900F5CF00F00900F5CF01F00900F5CF14
:1034700002F00900F5CF03F01200800ED819006E9B
:10348000800E6E0A005CD8A0C6D0640E046ED8C34D
:1034900000F078EC32F0120E0026000E00BEFF0E97
:1034A000016E000E0122020E046E000E01BEFF0E20
:1034B000026E036E0450000107E0003600900136F2
:1034C00002360336FF0FF7D700016E0E0026770E87
:1034D0000122000E022200C0F6FF01C0F7FF02C069
:1034E000F8FF0900F5CFD9F30900F5CFDAF30900A9
:1034F000F5CFDBF30900F5CFDCF3640E046ED8C31F
:1035000000F078EC32F008C000F00A0E046E78EC9F
:1035100032F0090E0026000E00BEFF0E016E000EF6
:103520000122020E046E000E01BEFF0E026E036E3B
:103530000450000107E000360090013602360336E1
:10354000FF0FF7D700016E0E0026770E0122000E46
:10355000022200C0F6FF01C0F7FF02C0F8FF090019
:10356000F5CF00F00900F5CF01F00900F5CF02F02A
:103570000900F5CF03F0D9C304F0DAC305F0DBC3CB
:1035800006F0DCC307F017EC2EF000C0D9F301C041
:10359000DAF302C0DBF303C0DCF30A0E046ED8C317
:1035A00000F078EC32F008C000F0020E046E000E5D
:1035B00000BEFF0E016E026E036E0450000107E0B4
:1035C00000360090013602360336FF0FF7D70001B0
:1035D0006E0E0026770E0122000E022200C0F6FFBA
:1035E00001C0F7FF02C0F8FF0900F5CF00F00900A5
:1035F000F5CF01F00900F5CF02F00900F5CF03F097
:10360000D9C304F0DAC305F0DBC306F0DCC307F06E
:1036100017EC2EF01200800E0A0A006E800E0301D5
:10362000D819005C76E20A0E046ED8C300F078EC7C
:1036300032F0090E0026000E00BEFF0E016E000ED5
:103640000122020E046E000E01BEFF0E026E036E1A
:103650000450000107E000360090013602360336C0
:10366000FF0FF7D700016E0E0026770E0122000E25
:10367000022200C0F6FF01C0F7FF02C0F8FF0900F8
:10368000F5CFD9F30900F5CFDAF30900F5CFDBF375
:103690000900F5CFDCF30A0E046ED8C300F078EC15
:1036A00032F008C000F0020E046E000E00BEFF0EE5
:1036B000016E026E036E0450000107E000360090B8
:1036C000013602360336FF0FF7D700016E0E0026D3
:1036D000770E0122000E022200C0F6FF01C0F7FFA4
:1036E00002C0F8FF0900F5CF00F00900F5CF01F0A6
:1036F0000900F5CF02F00900F5CF03F0D9C304F0BB
:10370000DAC305F0DBC306F0DCC307F017EC2EF0DC
:1037100012000001020E046ED8C300F0000E030177
:10372000D8BFFF0E016E026E036E0450030107E066
:1037300000360090013602360336FF0FF7D76E0EC3
:103740000026770E0122000E022200C0F6FF01C003
:10375000F7FF02C0F8FF0900F5CF00F00900F5CF30
:1037600001F00900F5CF02F00900F5CF03F01200D7
:103770000301546B556B4DC370F34EC371F34FC3CC
:1037800072F3EFEC30F0552B005203E0320E555D32
:10379000F2E3320E555D03E3FF0E006E1200DCEC27
:1037A00035F061C2D8F362C2D9F363C2DAF364C2FE
:1037B000DBF32A0E0301DC6F000EDD6FD3EC32F079
:1037C00002012851550AD8A467D02951AA0AD8A4C1
:1037D00063D02A50E90A09E02A50EB0A03E12C5091
:1037E000900A03E00201006A03D00201010E006E9C
:1037F00000524FE10101F45306E1F55304E1F653A1
:1038000002E1F75309E0F0C161F2F1C162F2F2C1E5
:1038100063F2F3C164F237D00201045306E10553A9
:1038200004E1065302E1075309E000C261F201C25C
:1038300062F202C263F203C264F225D0145306E1BD
:10384000155304E1165302E1175309E010C261F267
:1038500011C262F212C263F213C264F214D0245392
:1038600006E1255304E1265302E1275309E020C273
:1038700061F221C262F222C263F223C264F203D077
:10388000010E006E12000201020102010301546BDD
:1038900003D00301010E546F0301556B0301545310
:1038A00029E161C2D8F362C2D9F363C2DAF364C218
:1038B000DBF32A0EDC6F000EDD6FD3EC32F0020179
:1038C0002851550A07E12951AA0A04E1010E030112
:1038D000546F10D003015551400A03E1010E006EF0
:1038E0001200552B010E02016127000E6223632393
:1038F0006423D4D7010E0301556F5451010AD8A493
:103900006DD1080E046E36C000F0000E016E04503A
:10391000030105E0003600900136FF0FF9D70301DF
:10392000355000105E6F01C05FF3000E5F135EC381
:103930002AF25FC32BF237C038F2080E046E39C08A
:1039400000F0000E016E0450030105E00036009007
:103950000136FF0FF9D70301385000105C6F01C02A
:103960005DF3000E5D135CC358F25DC359F23AC0BB
:103970005FF2080E046E41C000F0000E016E0450AC
:10398000030105E0003600900136FF0FF9D703016F
:10399000405000105A6F01C05BF3000E5B135AC316
:1039A0005AF25BC35BF23AC000F0000E016E5AC3DC
:1039B00004F05BC305F094EC38F0000E026E036E69
:1039C00002016151002662510122635102226451B9
:1039D000032203015C510024566F5D510120576F93
:1039E000000E0220586F000E0320596F56C344F298
:1039F00057C345F258C346F259C347F2080E046E46
:103A00003CC000F0000E016E0450030105E00036DA
:103A100000900136FF0FF9D703013B500012000E52
:103A2000011200C05CF201C05DF2000E026E036E76
:103A3000050E046E0450030107E0003600900136C5
:103A400002360336FF0FF7D703015E510024086EDC
:103A50005F510120096E000E02200A6E000E032045
:103A60000B6E010E046E000E056E066E076E08C02A
:103A700000F009C001F00AC002F00BC003F00450CE
:103A8000005E0550015A0650025A0750035A5EC3A1
:103A900004F05FC305F0000E066E076E8AEC2BF093
:103AA0000050030156250201396F015003015721CF
:103AB00002013A6F02500301582102013B6F03508B
:103AC0000301592102013C6F03015C510201612590
:103AD000006E03015D5102016221016E000E63213F
:103AE000026E000E6421036E00C026F001C027F0B4
:103AF00002C028F003C029F003015A51002402013A
:103B00002C6F03015B51012002012D6F000E02207A
:103B10002E6F000E03202F6F5EC332F25FC333F2AD
:103B200033333233339F4050411054E03E503D1008
:103B300005E03DC050F33EC051F308D04AC050F3F9
:103B40004BC051F34CC052F34DC053F350C300F07F
:103B500051C301F052C302F053C303F002013951C3
:103B6000005E3A51015A3B51025A3C51035A38C245
:103B700004F0000E056E066E076E6FEC23F000C0B9
:103B800050F301C051F302C052F303C053F3000ECF
:103B9000035C08E1000E025C05E10F0E015C02E12E
:103BA000F50E005C04E2010E0301556F12D0030113
:103BB000000E535D08E1000E525D05E1FF0E515D00
:103BC00002E1F50E505D02E2556B03D00301010ED8
:103BD000556F04D00301010E006E1200030155C39E
:103BE00000F012000001025006180E6E086A096A01
:103BF0000B6A03500764E6EF1EF006500A6E068E4D
:103C0000028E03500B6E0750036E000E0B6436EFEE
:103C10001EF00B50075ED8B4D7EF1EF0070E0764F6
:103C2000A5EF1EF0075E00C008F001C000F002C062
:103C300001F0026A074ED7EF1EF007647AEF1EF01C
:103C4000075E00C008F001C000F0016A074ED7EF20
:103C50001EF0076458EF1EF0075E00C008F0006A0F
:103C6000074ED7EF1EF007643FEF1EF00AC002F0C8
:103C700005C001F004C000F0086A03EF20F0030E55
:103C800007644AEF1EF0075E08380F0B086E074EF8
:103C9000D7EF1EF0D8900832074ED7EF1EF0D8901D
:103CA0000832074ED7EF1EF0D8900832D7EF1EF03B
:103CB000030E076469EF1EF0075E08380F0B086EED
:103CC0000038F00B082600380F0B006E074ED7EFB8
:103CD0001EF0D89000320832074ED7EF1EF0D89071
:103CE00000320832074ED7EF1EF0D890003208326B
:103CF000D7EF1EF0030E076491EF1EF0075E083841
:103D00000F0B086E0038F00B082600380F0B006E02
:103D10000138F00B002601380F0B016E074ED7EF6C
:103D20001EF0D890013200320832074ED7EF1EF055
:103D3000D890013200320832074ED7EF1EF0D890EB
:103D4000013200320832D7EF1EF0030E0764C2EFD3
:103D50001EF0075E08380F0B086E0038F00B0826BF
:103D600000380F0B006E0138F00B002601380F0BE6
:103D7000016E0238F00B012602380F0B026E074E5F
:103D8000D7EF1EF0D8900232013200320832074ECF
:103D9000D7EF1EF0D8900232013200320832074EBF
:103DA000D7EF1EF0D8900232013200320832096A91
:103DB000000E0EAECBEF1FF0081E001E011E021EED
:103DC000082A002201220222CBEF1FF00750D8A4BC
:103DD000ECEF1EF003EF20F0096A02C00AF0028E39
:103DE000068E0750035C076ED8B4BEEF1FF0070EB7
:103DF00007648CEF1FF0075E0450096E0550046ED7
:103E00000650056E066A074EBEEF1FF0070E0764E8
:103E100061EF1FF0075E0450096E0550046E056ADD
:103E2000074EBEEF1FF0070E07643FEF1FF0075E5F
:103E30000450096E046A074EBEEF1FF0070E0764B8
:103E400026EF1FF00AC002F003EF20F0030E076414
:103E500031EF1FF0075E09380F0B096E074EBEEFFA
:103E60001FF0D8900932074EBEEF1FF0D8900932EC
:103E7000074EBEEF1FF0D8900932BEEF1FF0030EC1
:103E8000076450EF1FF0075E09380F0B096E043806
:103E9000F00B092604380F0B046E074EBEEF1FF01F
:103EA000D89004320932074EBEEF1FF0D89004328A
:103EB0000932074EBEEF1FF0D89004320932BEEF30
:103EC0001FF0030E076478EF1FF0075E09380F0B31
:103ED000096E0438F00B092604380F0B046E053800
:103EE000F00B042605380F0B056E074EBEEF1FF0D2
:103EF000D890053204320932074EBEEF1FF0D89039
:103F0000053204320932074EBEEF1FF0D890053259
:103F100004320932BEEF1FF0030E0764A9EF1FF051
:103F2000075E09380F0B096E0438F00B09260438B8
:103F30000F0B046E0538F00B042605380F0B056EC9
:103F40000638F00B052606380F0B066E074EBEEF3F
:103F50001FF0D8900632053204320932074EBEEF08
:103F60001FF0D8900632053204320932074EBEEFF8
:103F70001FF0D8900632053204320932086A000E6A
:103F80000EAECBEF1FF0091E041E051E061E092AE9
:103F9000042205220622095008260450002205505A
:103FA0000122065002220EBEE2EF1FF0D8A0F1EF70
:103FB0001FF00232013200320832033EF1EF1FF0EF
:103FC000FDEF1FF0D8B0F7EF1FF0000E081E001E27
:103FD000011E021E082A0022012202220A7EF7EF99
:103FE0001FF0010E0C6EABEC28F005EF20F0020E76
:103FF0000C6EABEC28F005EF20F0040E0C6E2AECF2
:104000003BF005EF20F0000E0C6E12000301506B28
:10401000516B50514D25E96E000E4E21EA6EEECFE8
:1040200002F00250000A49E050514D25E96E000EA1
:104030004E21EA6EEECF02F002502E0A02E150C38A
:1040400051F350514D25E96E000E4E21EA6EEECF30
:1040500070F3E2EC3AF00050011019E0550E616F78
:10406000030E626F50516127D8B0622B50514D251D
:10407000E96E000E4E21EA6EEECF70F350EC3BF08D
:1040800061C3E1FF62C3E2FF00C0E6FF13D0550E3B
:10409000E16E030EE26E03015051E126D8B0E22A30
:1040A00050514D25E96E000E4E21EA6EEECF00F024
:1040B00000C0E6FF0301502BACD7550EE16E030E96
:1040C000E26E5051E126D8B0E22AE66A515359E037
:1040D00051C350F3030E5125026E036A000E0322F2
:1040E000800E006E800E0318005C02E10250505DED
:1040F00048E25051010F006E016A000E0122550E78
:104100000024E96E030E0120EA6EEECF02F00250A9
:10411000000A1DE1020E5125026E036A000E032201
:10412000800E0318006E800E005C02E15051025CAC
:104130000CE3550EE16E030EE26E5051E126D8B04D
:10414000E22A200EE66E502BE5D703011AD0550E59
:10415000E16E030EE26E5051E126D8B0E22A5051D2
:10416000010F006E016A000E0122550E0024E96E57
:10417000030E0120EA6EEECF00F000C0E6FF502BE8
:10418000A9D7030150070A0E505D2FE2550EE96EC4
:10419000030EEA6E5051E926D8B0EA2AEECF5FF35B
:1041A0005007550EE96E030EEA6E5051E926D8B05D
:1041B000EA2AEECF5EF35007550EE96E030EEA6E63
:1041C0005051E926D8B0EA2AEECF5DF350510708E6
:1041D0000CE3550EE16E030EE26E5051E126D8B0AD
:1041E000E22A200EE66E502BF1D7606B02014A6B7B
:1041F0004B6B486B496B44C2D8F345C2D9F346C2F6
:10420000DAF347C2DBF32A0E0301DC6F000EDD6F29
:10421000D3EC32F00301526B536B516B02014B51E3
:104220002B1902E12A514A191DE14A6B4B6B484B8D
:10423000492B485144250301D86F020149514521BA
:104240000301D96F000E020146210301DA6F000E4F
:10425000020147210301DB6F2A0EDC6F000EDD6FC8
:10426000D3EC32F00301516B506B50510A0820E33C
:10427000505102014A25006E000E4B21016E2A0E9C
:104280000024E96E000E0120EA6EEECF04F0550E18
:10429000E96E030EEA6E03015051E926D8B0EA2A0E
:1042A000EECF02F004500218D8B4512B502BDDD7BA
:1042B000524B532B2A0E02014A25E96E000E4B2168
:1042C000EA6EEECF54F3200E4A27000E4B23030173
:1042D00051510B0A11E0535102015D1903E15C5188
:1042E00003015219030102E11E0E516F03015451E3
:1042F000000A02E1190E516F51510A088FE2140EA3
:10430000515D49E2200E02014A5D006E000E4B59DC
:10431000016E00C04AF201C04BF21A0E0026000ED8
:1043200001222A0E0024E96E000E0120EA6EEECF73
:1043300030F2EECF31F2BDEC38F01C0E4A25006EA3
:10434000000E4B21016E2A0E0024E96E000E0120A2
:10435000EA6EEECF50F2EECF51F2EECF52F2EECF48
:1043600053F2C1EC34F00E0E02014A25006E000E2D
:104370004B21016E2A0E0024E96E000E0120EA6E28
:10438000EECF67F2EECF68F2EECF65F2EECF66F2D7
:10439000010E006E120003014FAF0CD0550E706F6E
:1043A000030E716F7F0E4F15726F97EC2AF0010E9E
:1043B000006E1200006A12006E0E0301D85DD8A0D4
:1043C000D0D0640E046ED8C300F0D0EC3AF0120ED8
:1043D0000026016A000E0122020E046E000E01BECC
:1043E000FF0E026E036E0450000107E000360090DD
:1043F000013602360336FF0FF7D700013A0E0026CA
:10440000770E0122000E022200C0F6FF01C0F7FF66
:1044100002C0F8FF0900F5CF00F00900F5CF01F068
:104420000900F5CF02F00900F5CF03F0000E046E8D
:10443000000E056E000E066E7E0E076E17EC2EF057
:1044400000C0D9F301C0DAF302C0DBF303C0DCF330
:10445000640E046ED8C300F0D0EC3AF008C000F04F
:104460000A0E046ED0EC3AF0090E0026016A000E26
:104470000122020E046E000E01BEFF0E026E036EDC
:104480000450000107E00036009001360236033682
:10449000FF0FF7D700013A0E0026770E0122000E1B
:1044A000022200C0F6FF01C0F7FF02C0F8FF0900BA
:1044B000F5CF00F00900F5CF01F00900F5CF02F0CB
:1044C0000900F5CF03F0D9C304F0DAC305F0DBC36C
:1044D00006F0DCC307F017EC2EF000C0D9F301C0E2
:1044E000DAF302C0DBF303C0DCF30A0E046ED8C3B8
:1044F00000F0D0EC3AF008C000F0020E046E000E9E
:10450000016E026E036E0450000107E00036009059
:10451000013602360336FF0FF7D700013A0E0026A8
:10452000770E0122000E022200C0F6FF01C0F7FF45
:1045300002C0F8FF0900F5CF00F00900F5CF01F047
:104540000900F5CF02F00900F5CF03F0D9C304F05C
:10455000DAC305F0DBC306F0DCC307F017EC2EF07E
:1045600012000301D8510A08D8B083D00A0E046E95
:10457000D8C300F0D0EC3AF0090E0026016A000E14
:104580000122020E046E000E01BEFF0E026E036ECB
:104590000450000107E00036009001360236033671
:1045A000FF0FF7D700013A0E0026770E0122000E0A
:1045B000022200C0F6FF01C0F7FF02C0F8FF0900A9
:1045C000F5CF00F00900F5CF01F00900F5CF02F0BA
:1045D0000900F5CF03F0000E046E000E056E000E0C
:1045E000066E7E0E076E17EC2EF000C0D9F301C0E8
:1045F000DAF302C0DBF303C0DCF30A0E046ED8C3A7
:1046000000F0D0EC3AF008C000F0020E046E000E8C
:10461000016E026E036E0450000107E00036009048
:10462000013602360336FF0FF7D700013A0E002697
:10463000770E0122000E022200C0F6FF01C0F7FF34
:1046400002C0F8FF0900F5CF00F00900F5CF01F036
:104650000900F5CF02F00900F5CF03F0D9C304F04B
:10466000DAC305F0DBC306F0DCC307F017EC2EF06D
:1046700012000001020E046ED8C300F0000E016E9D
:10468000026E036E0450000107E000360090013610
:1046900002360336FF0FF7D73A0E0026770E0122B7
:1046A000000E022200C0F6FF01C0F7FF02C0F8FFB3
:1046B0000900F5CF00F00900F5CF01F00900F5CFB2
:1046C00002F00900F5CF03F0000E046E000E056E37
:1046D000000E066E7E0E076E17EC2EF01200000123
:1046E0000B6A0A6A096A086A0E6A033408360450BB
:1046F000085E0550D8A0053C095E0650D8A0063CCF
:104700000A5E0750D8A0073C0B5EE86AD8A0010EED
:104710000E5E0336070E0C6E0334083609360A3671
:104720000B360E36045003A0A9EF23F0085E0550A7
:10473000D8A0053C095E0650D8A0063C0A5E07508A
:10474000D8A0073C0B5EE86AD8A0010E0E5EBAEF57
:1047500023F008260550D8B0053C09260650D8B0ED
:10476000063C0A260750D8B0073C0B26E86AD8B0AA
:10477000010E0E2603360C2E8CEF23F00234083681
:1047800009360A360B360E36045003A0DBEF23F051
:10479000085E0550D8A0053C095E0650D8A0063C2E
:1047A0000A5E0750D8A0073C0B5EE86AD8A0010E4D
:1047B0000E5EECEF23F008260550D8B0053C092624
:1047C0000650D8B0063C0A260750D8B0073C0B2646
:1047D000E86AD8B0010E0E260236070E0C6E0234BF
:1047E000083609360A360B360E36045002A00CEF96
:1047F00024F0085E0550D8A0053C095E0650D8A0FC
:10480000063C0A5E0750D8A0073C0B5EE86AD8A0B9
:10481000010E0E5E1DEF24F008260550D8B0053CB1
:1048200009260650D8B0063C0A260750D8B0073CE7
:104830000B26E86AD8B0010E0E2602360C2EEFEFDA
:1048400023F00134083609360A360B360E3604508A
:1048500002A03EEF24F0085E0550D8A0053C095E9A
:104860000650D8A0063C0A5E0750D8A0073C0B5E55
:10487000E86AD8A0010E0E5E4FEF24F0082605501E
:10488000D8B0053C09260650D8B0063C0A26075089
:10489000D8B0073C0B26E86AD8B0010E0E260136C8
:1048A000070E0C6E0134083609360A360B360E3602
:1048B000045001A06FEF24F0085E0550D8A0053C1D
:1048C000095E0650D8A0063C0A5E0750D8A0073CF7
:1048D0000B5EE86AD8A0010E0E5E80EF24F0082679
:1048E0000550D8B0053C09260650D8B0063C0A262B
:1048F0000750D8B0073C0B26E86AD8B0010E0E2648
:1049000001360C2E52EF24F00034083609360A36F0
:104910000B360E36045001A0A1EF24F0085E0550BE
:10492000D8A0053C095E0650D8A0063C0A5E075098
:10493000D8A0073C0B5EE86AD8A0010E0E5EB2EF6D
:1049400024F008260550D8B0053C09260650D8B0FA
:10495000063C0A260750D8B0073C0B26E86AD8B0B8
:10496000010E0E260036070E0C6E0034083609368E
:104970000A360B360E36045000A0D2EF24F0085E43
:104980000550D8A0053C095E0650D8A0063C0A5E3A
:104990000750D8A0073C0B5EE86AD8A0010E0E5E57
:1049A000E3EF24F008260550D8B0053C0926065050
:1049B000D8B0063C0A260750D8B0073C0B26E86A58
:1049C000D8B0010E0E2600360C2EB5EF24F000B044
:1049D000F8EF24F0045008260550D8B0053C09260D
:1049E0000650D8B0063C0A260750D8B0073C0B2624
:1049F00012007FEC39F02D0E0301326F530E336F2E
:104A00004F0E346F4C0E356F410E366F520E376FAE
:104A1000200E386F520E396F450E3A6F430E3B6FC2
:104A20004F0E3C6F520E3D6F440E3E6F450E3F6F72
:104A3000520E406F2D0E416F426B4E0E436F6F0E44
:104A4000446F200E456F4D0E466F4D0E476F430E5F
:104A5000486F2F0E496F530E4A6F440E4B6F4C6BCD
:104A6000836A956A800EC16EFF0E926E080E966E76
:104A7000850ED56EA00EF26E020E0C6EFF0E0B6E42
:104A8000FF0E0A6E0C2E01D007D00B2E01D003D0E2
:104A90000A2EFED7FAD7F6D7060E0B6EFF0E0A6E59
:104AA0000B2E01D003D00A2EFED7FAD70A0E0A6EBB
:104AB0000A2EFED7810E4D6F0F0E4E6FA8EC2FF011
:104AC000010E0301D86F74EC34F00C0E0301D86FA3
:104AD00074EC34F0010E0301AF6F010EB06F320EB3
:104AE000B16F030EB26F09EC35F00B0E0C6EFF0EBA
:104AF0000B6EFF0E0A6E0C2E01D007D00B2E01D0CC
:104B000003D00A2EFED7FAD7F6D7330E0B6EFF0E60
:104B10000A6E0B2E01D003D00A2EFED7FAD7880ECC
:104B20000A6E0A2EFED7830E4D6F0F0E4E6FA9EC44
:104B30003AF095EC3AF0010E0301706FE5EC38F0B5
:104B4000000E015C02E1640E005C02E2D3EC33F083
:104B5000DBEC36F0010E03014D6F4E6B4F6B010E17
:104B6000506F40EC3AF0010ED86F74EC34F02BEC3F
:104B70002FF0820E0301706F0F0E716F020E726FB5
:104B8000EFEC30F000520DE0020EAF6F010EB06F8F
:104B9000430EB16F030EB26F09EC35F0DBEC36F06B
:104BA000E8D72C6B2D6B02013D6B010E0301D86F12
:104BB00074EC34F05FEC36F0820E03014D6F0F0E93
:104BC0004E6F020E4F6FB8EC1BF0960E03014D6F47
:104BD000020E4E6FA00E4F6F06EC20F0AC0E0301DC
:104BE0004D6F020E4E6F960E4F6F020E506F33ECEC
:104BF00039F0200E0201B46F200EB56F200EB66F93
:104C0000010E0301AF6F010EB06FAC0EB16F020E5B
:104C1000B26F09EC35F0010ED16E195235E0A9ECF6
:104C200027F079EC37F02AEC33F0AC0E03014D6F2E
:104C3000020E4E6FF5EC39F000C04FF301C050F397
:104C4000AC0E4D6F020E4E6FA1EC29F0AC0E0301BD
:104C50004D6F020E4E6FA00E4F6F780E506F000E0C
:104C6000516F2CC352F32DC353F30DEC39F0010EE9
:104C7000AF6F0C0EB06FAC0EB16F020EB26F09ECDD
:104C800035F0DBEC36F0196A040079EC37F07FEC94
:104C900033F0020E0C6EFF0E0B6EFF0E0A6E0C2E22
:104CA00001D007D00B2E01D003D00A2EFED7FAD7A1
:104CB000F6D7060E0B6EFF0E0A6E0B2E01D003D038
:104CC0000A2EFED7FAD70A0E0A6E0A2EFED7A5D7ED
:104CD000FFD700010450085E0550D8A0053C095ECE
:104CE0000650D8A0063C0A5E0750D8A0073C0B5ED1
:104CF0000336070E0C6E0334083609360A360B36B7
:104D0000045003A093EF26F0085E0550D8A0053CA0
:104D1000095E0650D8A0063C0A5E0750D8A0073CA2
:104D20000B5EA0EF26F008260550D8B0053C0926FA
:104D30000650D8B0063C0A260750D8B0073C0B26D0
:104D400003360C2E7BEF26F00234083609360A367D
:104D50000B36045003A0BCEF26F0085E0550D8A027
:104D6000053C095E0650D8A0063C0A5E0750D8A054
:104D7000073C0B5EC9EF26F008260550D8B0053C6D
:104D800009260650D8B0063C0A260750D8B0073C82
:104D90000B260236070E0C6E0234083609360A3628
:104DA0000B36045002A0E4EF26F0085E0550D8A0B0
:104DB000053C095E0650D8A0063C0A5E0750D8A004
:104DC000073C0B5EF1EF26F008260550D8B0053CF5
:104DD00009260650D8B0063C0A260750D8B0073C32
:104DE0000B2602360C2ECCEF26F00134083609369D
:104DF0000A360B36045002A00DEF27F0085E05506E
:104E0000D8A0053C095E0650D8A0063C0A5E0750B3
:104E1000D8A0073C0B5E1AEF27F008260550D8B043
:104E2000053C09260650D8B0063C0A260750D8B0E3
:104E3000073C0B260136070E0C6E01340836093686
:104E40000A360B36045001A035EF27F0085E0550F6
:104E5000D8A0053C095E0650D8A0063C0A5E075063
:104E6000D8A0073C0B5E42EF27F008260550D8B0CB
:104E7000053C09260650D8B0063C0A260750D8B093
:104E8000073C0B2601360C2E1DEF27F000340836A8
:104E900009360A360B36045001A05EEF27F0085E93
:104EA0000550D8A0053C095E0650D8A0063C0A5E15
:104EB0000750D8A0073C0B5E6BEF27F00826055083
:104EC000D8B0053C09260650D8B0063C0A26075043
:104ED000D8B0073C0B260036070E0C6E003408369F
:104EE00009360A360B36045000A086EF27F0085E1C
:104EF0000550D8A0053C095E0650D8A0063C0A5EC5
:104F00000750D8A0073C0B5E93EF27F0082605500A
:104F1000D8B0053C09260650D8B0063C0A260750F2
:104F2000D8B0073C0B2600360C2E6EEF27F000B0F1
:104F3000A8EF27F0045008260550D8B0053C0926F4
:104F40000650D8B0063C0A260750D8B0073C0B26BE
:104F50001200225026240301D86F23502720D96F36
:104F6000000E2820DA6F000E2920DB6F2A0EDC6F7E
:104F7000000EDD6FD3EC32F02A0E2424E96E000E11
:104F80002520EA6EEECF4DF3000E03014E6F4F6FFA
:104F9000506F000E4E6F4F6F506FEECF4EF3030108
:104FA000000E006E501908E100504F1905E1FF0E88
:104FB0004E1902E14D51FF0A6DE04DC355F34EC34A
:104FC00056F34FC357F350C358F3553755915637DF
:104FD0005737583755C34DF356C34EF357C34FF3A6
:104FE00058C350F32AC204F02BC205F0000E066E1F
:104FF000076E55C300F056C301F057C302F058C303
:1050000003F06FEC23F000C051F301C052F302C073
:1050100053F303C054F351C322F052C323F02AC206
:1050200004F02BC205F0000E066E076E55C300F0AB
:1050300056C301F057C302F058C303F06FEC23F0DE
:1050400008C000F009C001F00AC002F00BC003F074
:1050500000C024F001C025F0030151512624D86F6F
:1050600052512720D96F000E2820DA6F000E292018
:10507000DB6F2A0EDC6F000EDD6FD3EC32F02A0EF0
:105080002424E96E000E2520EA6EEECF4DF3EECF1C
:105090004EF385D70FEC3AF0BDEC38F038C200F093
:1050A000000E016E026E036E2AC204F02BC205F0E0
:1050B000000E066E076E11EC37F000C004F001C060
:1050C00005F002C006F003C007F050C200F051C264
:1050D00001F052C202F053C203F06FEC23F008C09B
:1050E00000F009C001F00AC002F00BC003F02AC2B0
:1050F00004F02BC205F0000E066E076E6FEC23F075
:1051000000C05EF2005002013427000E3523362322
:1051100037232AC204F02BC205F0000E066E076E7C
:1051200050C200F051C201F052C202F053C203F06B
:105130006FEC23F008C000F009C001F00AC002F0D3
:105140000BC003F000C04CF201C04DF202C04EF2A1
:1051500003C04FF2120000010CB0EEEF28F00CA2D9
:1051600096EF29F00E6A000E026405EF29F0F00EAA
:105170000214D8A4D0EF28F0023A01380F0B02260F
:105180000138F00B016E00380F0B01260038F00BD0
:10519000006E08380F0B00260838F00B086E0E84DE
:1051A000D89002BEE9EF28F0083600360136023604
:1051B0000E2A02BEE9EF28F0083600360136023624
:1051C0000E2A02BEE9EF28F0083600360136023614
:1051D0000E2A0E5003648AEF29F0035E0BBC08AE62
:1051E00090EF29F0D880800E08640030000E002275
:1051F00001220222D8A090EF29F0023201320032BF
:10520000034A96EF29F090EF29F001C002F000C0A8
:1052100001F008C000F0086A000E0E8602643CEF40
:1052200029F0F00E0214D8A424EF29F0023A013834
:105230000F0B02260138F00B016E00380F0B012610
:105240000038F00B006E0E84D89002BEE9EF28F013
:105250000036013602360E2A02BEE9EF28F000368B
:10526000013602360E2A02BEE9EF28F0003601367A
:1052700002360E2AE9EF28F001C002F000C001F06A
:10528000006A000E0E960E88026469EF29F0F00E97
:105290000214D8A454EF29F0023A01380F0B022669
:1052A0000138F00B016E0E84D89002BEE9EF28F0B1
:1052B000013602360E2A02BEE9EF28F00136023628
:1052C0000E2A02BEE9EF28F0013602360E2AE9EF77
:1052D00028F001C002F0016A000E0E8602649CEF05
:1052E00029F0F00E0214D8A478EF29F0023A0E84C7
:1052F000D89002BEE9EF28F002360E2A02BEE9EF8E
:1053000028F002360E2A02BEE9EF28F002360E2AF5
:10531000E9EF28F0010E0C6E0FEC3BF0A0EF29F046
:10532000020E0C6E87EC3BF0A0EF29F0040E0C6E21
:105330002AEC3BF0A0EF29F0080E0C6E5BEC3BF082
:10534000120034C2D8F335C2D9F336C2DAF337C209
:10535000DBF32A0E0301DC6F000EDD6FD3EC32F0BD
:105360000301516B526B5051525D02E14F51515D3F
:105370005AE22A0E02014C25E16E000E4D21E26E2A
:10538000030151514D25E96E52514E21EA6EEECF87
:1053900000F000C0E6FF010E02014C27000E4D2375
:1053A0004E234F23000E006E4F1908E100504E1996
:1053B00005E12B514D1902E14C512A1930E134C25B
:1053C000D8F335C2D9F336C2DAF337C2DBF32A0E8B
:1053D0000301DC6F000EDD6FABEC2EF0010E02015D
:1053E0003427000E3523362337234C6B4D6B4E6B21
:1053F0004F6B5E2B5E51381903E15E6BB7EC31F0F9
:1054000034C2D8F335C2D9F336C2DAF337C2DBF38C
:105410002A0E0301DC6F000EDD6FD3EC32F00301C6
:10542000514B522BA0D7030134C2D8F335C2D9F364
:1054300036C2DAF337C2DBF32A0EDC6F000EDD6F03
:10544000ABEC2EF0030151510201502703015251E0
:1054500002015123000E52235323485144250301D6
:10546000D86F0201495145210301D96F000E020195
:1054700046210301DA6F000E020147210301DB6FB1
:105480002A0EDC6F000EDD6FD3EC32F00E0E02013F
:105490004A25006E000E4B21016E2A0E0024E16E9B
:1054A000000E0120E26E67C2E6FF68C2E6FF65C239
:1054B000E6FF66C2E6FF65C2E6FF66C2E6FFE66A91
:1054C000E66A67C2E6FF68C2E6FF65C2E6FF66C23B
:1054D000E6FF1C0E4A25006E000E4B21016E2A0EBF
:1054E0000024E16E000E0120E26E50C2E6FF51C2C0
:1054F000E6FF52C2E6FF53C2E6FF485144250301CE
:10550000D86F0201495145210301D96F000E0201F4
:1055100046210301DA6F000E020147210301DB6F10
:105520002A0EDC6F000EDD6FABEC2EF012000201D4
:105530004A6B4B6B486B496B18EC32F098EC35F0CA
:105540000FEC3AF044C2D8F345C2D9F346C2DAF3BD
:1055500047C2DBF32A0E0301DC6F000EDD6FD3ECD4
:1055600032F00301746B02014B512B1902E12A51F5
:105570004A191DE14A6B4B6B484B492B4851442556
:105580000301D86F0201495145210301D96F000E73
:10559000020146210301DA6F000E020147210301D7
:1055A000DB6F2A0EDC6F000EDD6FD3EC32F02A0EBB
:1055B00002014A25E96E000E4B21EA6EEECF02F0A1
:1055C0000250E50A0BE02A0E4A25E96E000E4B2137
:1055D000EA6EEECF02F00250000A03E1010E030171
:1055E000746F200E02014A27000E4B2303017453EF
:1055F000BAE07451010AD8A48AD0200E02014A5F91
:10560000000E4B5B0301736B73510A081AE373516D
:1056100002014A25006E000E4B21016E2A0E002465
:10562000E16E000E0120E26E030173517025E96EF8
:10563000000E7121EA6EEECF00F000C0E6FF732B82
:10564000E3D71C0E736F200E735D11E273510201DC
:105650004A25006E000E4B21016E2A0E0024E16ED9
:10566000000E0120E26EE66A0301732BECD71A0EDE
:1056700002014A25006E000E4B21016E2A0E002405
:10568000E16E000E0120E26E30C2E6FF31C2E6FF9D
:105690000B0E4A25006E000E4B21016E2A0E0024CF
:1056A000E16E000E0120E26E72C3E6FF0D0E0301F3
:1056B000736F7351190811E3735102014A25006E8B
:1056C000000E4B21016E2A0E0024E16E000E012017
:1056D000E26EE66A0301732BECD7020148514425C0
:1056E0000301D86F0201495145210301D96F000E12
:1056F000020146210301DA6F000E02014721030176
:10570000DB6F2A0EDC6F000EDD6FABEC2EF0BDEC14
:1057100038F0120000010C6A07BE0C2A0D6A0B6AF1
:105720000A6A096A086A0350021001100010D8B40E
:105730002EEF2CF0035007180E6E0EBE0D1E07AE96
:10574000ADEF2BF0041E051E061E071E042AD8B45A
:10575000052AD8B4062AD8B4072A03AEBBEF2BF02B
:10576000001E011E021E031E002AD8B4012AD8B44E
:10577000022AD8B4032A035007100E6E0EBEE1EFC2
:105780002BF069EC26F00CBE02EF2CF00DAE2EEFE4
:105790002CF0001E011E021E031E002AD8B4012A8E
:1057A000D8B4022AD8B4032A081E091E0A1E0B1EEA
:1057B000082AD8B4092AD8B40A2AD8B40B2A2EEF5A
:1057C0002CF007AEFBEF2BF003BEF5EF2BF00350F0
:1057D0000B6E02500A6E0150096E0050086E036A8B
:1057E000026A016A006AC6EF2BF0036A026A016A64
:1057F000006A002A000C031E021E011E001E0C8EF1
:10580000C1EF2BF0082AD8B4092AD8B40A2AD8B490
:105810000B2A0450085CD8A4C6EF2BF00550095C95
:10582000D8A4C6EF2BF006500A5CD8A4C6EF2BF024
:1058300007500B5CD8A4C6EF2BF00B6A0A6A096A02
:10584000086A002AD8B4012AD8B4022AD8B4032A94
:1058500003AEC6EF2BF00E6A0E88FF0C0E6A0CA08A
:1058600034EF2CF01DEC3BF0000F12000001086A31
:10587000096A0750D8B4CDEF2CF00350D8B4D2EF5A
:105880002CF0025006180A6E028E068E0E6A02C0B6
:1058900008F001C00CF000C00DF004500D5E055082
:1058A000D8A0053C0C5E0650D8A0063C085E086AED
:1058B0000C6A0D6AD8A064EF2CF0D8900232013245
:1058C00000320832010E0E6E0750035ED8A071EF51
:1058D0002CF07E0E0E240326D8B0D7EF2CF077EFF5
:1058E0002CF07E0E0E240326D8A0DCEF2CF0180E30
:1058F0000B6E0D360C3608360036013602360E3683
:105900000450005E0550D8A0053C015E0650D8A0AA
:10591000063C025E06340E120EA092EF2CF00D80B3
:105920009DEF2CF0045000260550D8B0053C012610
:105930000650D8B0062802260D900B2E79EF2CF0D9
:10594000C3EF2CF0D8900036013602360E360450E4
:10595000005E0550D8A0053C015E0650D8A0063C6C
:10596000025E06340E10010B0D26D8B00C2AD8B4F6
:10597000082AD8A4C3EF2CF008320C320D32032AC7
:10598000D8B4D7EF2CF00AAE089E0850026E0C5027
:10599000016E0D50006EDFEF2CF0010E96EC3BF027
:1059A000DFEF2CF0020E5BEC3BF0DFEF2CF0040E8F
:1059B0002AEC3BF0DFEF2CF0080E0FEC3BF012006E
:1059C00000010B6A0C6A0A6A086A0350D8B469EFCE
:1059D0002DF0028E9E0E035E03BEF4EF2CF0D8B4C1
:1059E000F4EF2CF059EF2DF0036C080E035CD8A0F7
:1059F00026EF2DF0036E083600C008F001C000F05D
:105A000002C001F0026A080E035CD8A026EF2DF058
:105A1000036E083600C008F001C000F0016A080EED
:105A2000035CD8A026EF2DF0036E083600C008F006
:105A3000006A080E035CD8A026EF2DF0036E08362E
:105A4000086A0350D8A4D89032EF2DF00350D8B490
:105A500032EF2DF0D8900232013200320832032E9C
:105A60002AEF2DF00BBC08A043EF2DF0D8A043EF98
:105A70002DF0082AD8B4002AD8B4012AD8B4022AB2
:105A800002BE6DEF2DF00AAE69EF2DF0021E011E71
:105A9000001E081E082AD8B4002AD8B4012AD8B497
:105AA000022A69EF2DF0026A016A006A086A69EF4A
:105AB0002DF00B800BAE73EF2DF0026A0AAE73EF80
:105AC0002DF0026E016E006E086E0A36023273EF20
:105AD0002DF0000E0C6A74EF2DF0010E0C6E00EC30
:105AE0003BF074EF2DF0FF0E0250036E0150026E7A
:105AF0000050016E0850006E120000010B6A0C6A23
:105B0000086A0350D8B402EF2EF002C00AF0028EE9
:105B10009E0E035E03AEF2EF2DF0036C080E035CE5
:105B2000D8A0BFEF2DF0036E083600C008F001C00A
:105B300000F002C001F0026A080E035CD8A0BFEFBB
:105B40002DF0036E083600C008F001C000F0016AB5
:105B5000080E035CD8A0BFEF2DF0036E083600C01E
:105B600008F0006A080E035CD8A0BFEF2DF0036EAA
:105B70000836086A0350D8A4D890CBEF2DF0035014
:105B8000D8B4CBEF2DF0D890023201320032083277
:105B9000032EC3EF2DF00BBC08A0DCEF2DF0D8A036
:105BA000DCEF2DF0082AD8B4002AD8B4012AD8B4E2
:105BB000022A02BE06EF2EF00AAE02EF2EF0021EFF
:105BC000011E001E081E082AD8B4002AD8B4012AD3
:105BD000D8B4022A02EF2EF0026A016A006A086A4B
:105BE00002EF2EF00B800BAE0DEF2EF0026A0AAE24
:105BF0000DEF2EF0026E016E006E086E0A36023254
:105C00000DEF2EF00C6A000E0EEF2EF0010E0C6E52
:105C1000000E00EC3BF00EEF2EF0FF0E0250036E74
:105C20000150026E0050016E0850006E120000011B
:105C3000086A096A000E076203649DEF2EF00250A5
:105C400006180A6E075003267E0ED8A02EEF2EF0FF
:105C5000035ED8B0A2EF2EF032EF2EF0035ED8A094
:105C6000A7EF2EF0028E068E02C00EF001C00BF0E0
:105C700000C00DF000500402F4CF0CF001500502FA
:105C8000F4CF00F0F3CF08F00402F3500C26F450E8
:105C90000822000E00220D500502F3500C26F4508D
:105CA0000822000E002202500402F3500826F4508D
:105CB000002202500502016A000E0122F350002664
:105CC000F45001220D500602F3500826F450002231
:105CD000026A000E012202220B500602F350002637
:105CE000F4500122000E02220E500602F35001264B
:105CF000F450022202BE85EF2EF00836003601363F
:105D000002360306D8B4A7EF2EF098EF2EF0D88015
:105D1000800E08640030000E002201220222D8A06A
:105D200098EF2EF0023201320032034AA2EF2EF039
:105D30000AAE029E000EAAEF2EF0010E5BEC3BF0C5
:105D4000AAEF2EF0020E2AEC3BF0AAEF2EF0040E82
:105D50000FEC3BF0120073EC3BF0090E006ED8C361
:105D6000E3F3D9C3E4F3DAC3E5F3DBC3E6F30050AE
:105D700008E00301E337E391E437E537E637FF0F47
:105D8000F7D70301180EE26FFF0EE76F1EEC36F037
:105D9000005205E044EC3BF0010E006E1200FF0ED5
:105DA0000301EB6F7AEC3BF0FF0E0301EB6F7AEC33
:105DB0003BF0FE0E0301EB6F7AEC3BF00301DE6B70
:105DC000DF6BDF51010802E1DE51FF080EE3DE5117
:105DD000DC25E96EDF51DD21EA6EEECFEBF37AECE4
:105DE0003BF00301DE4BDF2BECD70301FF0EEB6F23
:105DF0007AEC3BF0FF0E0301EB6F7AEC3BF0FF0E09
:105E00000301EB6F7AEC3BF000C0DEF3000E030100
:105E1000DF6F1F0EDE15016EDFC302F0000E0216EB
:105E200001C0DEF302C0DFF3000E021802E1050E2E
:105E3000011805E044EC3BF0020E006E1200FF0E6C
:105E40000301EB6F7AEC3BF00050FF0AF8E144EC01
:105E50003BF0006A1200360E03014D6F300E4E6F9C
:105E6000200E4F6F730E506F650E516F630E526FA1
:105E70006F0E536F6E0E546F640E556F730E566F28
:105E8000576B310E586F300E596F200E5A6F730ECC
:105E90005B6F650E5C6F630E5D6F6F0E5E6F6E0EF7
:105EA0005F6F640E606F730E616F626B330E636FB2
:105EB000300E646F300E656F200E666F730E676F65
:105EC000650E686F630E696F6F0E6A6F6E0E6B6F93
:105ED000640E6C6F730E6D6F6E6B706B63EC3BF0EA
:105EE00000C06FF30050FF0A0FE13C0E176E000E6A
:105EF000186E010E0301AF6F010EB06F4D0EB16F42
:105F0000030EB26F09EC35F003016F51000A0EE188
:105F10000A0E176E000E186E010EAF6F010EB06FF5
:105F2000580EB16F030EB26F09EC35F06F51010AD4
:105F30000EE12C0E176E010E186E010EAF6F010EE2
:105F4000B06F630EB16F030EB26F09EC35F0120043
:105F50004DC31FF04EC320F01FC0E1FF20C0E2FF81
:105F6000120EE126E796E794E790E79EE79CE79A12
:105F7000E798120EE15EE796E794E790E79EE79CCC
:105F8000E79AE798F1EC3AF0E78AE788E7869BEC36
:105F90003BF0E796F1EC3AF0E78AE788E7869BEC7E
:105FA0003BF0E79681EC3BF081EC3BF0E78AE78839
:105FB000E7869BEC3BF0E796F1EC3AF0E78AE7984E
:105FC000E7869BEC3BF0E79681EC3BF0E78AE798AD
:105FD000E7869BEC3BF0E796E78EE79CE7869BEC39
:105FE0003BF0E79681EC3BF0000EE76EE7869BEC1A
:105FF0003BF0E796E78EE78CE78AE788E7869BEC3D
:106000003BF0E79681EC3BF0000EE76EE7869BECF9
:106010003BF0E796E788E7869BEC3BF0E796F1ECF0
:106020003AF0000EE76EE7869BEC3BF0E796E78CD4
:10603000E78AE7869BEC3BF0E79681EC3BF0010EAC
:10604000216E120000010A6A0350D8A40A8007508A
:10605000D8A40A820A50D8B486EF30F0030AD8B424
:106060003FEF30F00AB03AEF30F006AE84EF30F098
:1060700082EF30F002AE82EF30F084EF30F0025069
:10608000800B0A6E029E0650800B069E0A18D8B43A
:1060900050EF30F00A50D8B482EF30F084EF30F097
:1060A0000750035CD8B45AEF30F0D8A076EF30F048
:1060B0007CEF30F00650025CD8B464EF30F0D8A02A
:1060C00076EF30F07CEF30F00550015CD8B46EEF25
:1060D00030F0D8A076EF30F07CEF30F00450005C68
:1060E000D8B486EF30F0D8B07CEF30F00A52D8B494
:1060F00084EF30F082EF30F00A52D8B482EF30F003
:1061000084EF30F0D8801200D8901200D880D88464
:106110001200120000010D6A096A086A015000109D
:10612000D8B4000C015005180A6E0ABE0D1E0B6A89
:1061300005AEA0EF30F0041E051E042AD8B4052ACF
:1061400001AEA8EF30F0001E011E002AD8B4012ACB
:10615000015005100A6E0ABEC0EF30F0ABEC37F00C
:106160000BB0D7EF30F00DAE000C001E011E002A60
:10617000D8B4012A081E091E082AD8B4092A000C1E
:1061800005AED2EF30F001BECEEF30F00150096E17
:106190000050086E016A006AB3EF30F0016A006ACD
:1061A000002A000C011E001E0B2AAEEF30F0082A58
:1061B000D8B4092A0450085CD8A4B3EF30F00550D5
:1061C000095CD8A4B3EF30F0096A086A002AD8B491
:1061D000012A01AEB3EF30F00000FF0C120072C3D1
:1061E00000F0010E016E005004E001360190FF0F37
:1061F000FBD701C01DF0011C006E00C01CF0090E91
:10620000030170251A6E000E71211B6E1AC0E9FF82
:106210001BC0EAFF0150EF12090E1A24E96E00506C
:10622000EF16746B0A0E745D07E2FF0EEB6F7AECEB
:106230003BF00301742BF6D773EC3BF00301E26BE8
:10624000E36BE46BE56BE66B950EE76F1EEC36F0E7
:1062500000C074F344EC3BF003017451010A03E005
:10626000010E006E1200746BFF0E745D19E273EC88
:106270003BF0010E0301E26FE36BE46BE56BE66B51
:10628000FF0EE76F1EEC36F000C073F344EC3BF0FA
:1062900003017351000A02E1006A1200742BE4D773
:1062A000010E006E1200010E0301DA6F080ED96FA5
:1062B0001EC0E9FF0F0EEA6ED95324E09BEC3BF0C1
:1062C0009BEC3BF06BEC3BF0EF9C9BEC3BF0030159
:1062D000D85300E06BEC3BF0D837D8A073EF31F027
:1062E000EF8A74EF31F0EF9A00009BEC3BF0EF8CFB
:1062F000120EE95EEFAC7AEF31F0120EE9260301DF
:10630000D907DAD7DA6B9BEC3BF06BEC3BF0000083
:10631000EF9C9BEC3BF0EF8A9BEC3BF09BEC3BF063
:106320000301DA5300E0EF8C120EE95EEFAC96EF5A
:1063300031F0DA6B9BEC3BF0EFBADA819BEC3BF08F
:106340009BEC3BF09BEC3BF09BEC3BF09BEC3BF085
:106350009BEC3BF09BEC3BF09BEC3BF06BEC3BF0A5
:10636000120EE926EF9CEF9ADAC300F0120022C069
:1063700054F223C055F224C056F225C057F218EC4F
:1063800032F098EC35F00FEC3AF00201545126242B
:106390000301D86F0201555127200301D96F000E68
:1063A0002820DA6F000E2920DB6F2A0EDC6F000E2A
:1063B000DD6FD3EC32F02A0E02015625E16E000E9D
:1063C0005721E26E30C2E6FF31C2E6FF5451262467
:1063D0000301D86F0201555127200301D96F000E28
:1063E0002820DA6F000E2920DB6F2A0EDC6F000EEA
:1063F000DD6FABEC2EF0020154512C250301D86F58
:10640000020155512D210301D96F000E02012E21E9
:106410000301DA6F000E02012F210301DB6F2A0E48
:10642000DC6F000EDD6FABEC2EF0BDEC38F012002F
:106430000301AF6B226A236A040E246E000E256EE0
:1064400026C0D8F327C0D9F328C0DAF329C0DBF37C
:106450002A0EDC6F000EDD6FD3EC32F02550020106
:106460002B1902E12A51241817E1246A256A224ACD
:10647000232A225026240301D86F23502720D96FC6
:10648000000E2820DA6F000E2920DB6F2A0EDC6F49
:10649000000EDD6FD3EC32F02A0E2424E96E000EDC
:1064A0002520EA6EEECF02F00250000A14E1010E40
:1064B0002424006E000E2520016E2A0E0024E96EB1
:1064C000000E0120EA6EEECF02F00250000A03E156
:1064D000010E0301AF6F0301020E2426000E2522D8
:1064E000AF53BCE0AF6B020E245E000E255A1200C3
:1064F00000010D6A086A0050D8B4000C04180A6E36
:106500000ABE0D1E0B6A04AE88EF32F0041E042A88
:1065100000A08DEF32F0001E002A005004100A6E19
:106520000ABEB4EF32F00450085E0036003408367C
:10653000045008260036060E0C6E0034083604504F
:1065400000B0085E00A0082600360C2E9DEF32F049
:1065500000A008260BB0C6EF32F00DAE000C001EF6
:10656000002A081E082A000C04AEC2EF32F000BE5A
:10657000BFEF32F00050086E006AADEF32F0006AF3
:10658000002A000C001E0B2A93EF32F0082A045058
:10659000085CD8A4ADEF32F0086A002A00AEADEF77
:1065A00032F0FF0C120073EC3BF0090E006ED8C302
:1065B000E3F3D9C3E4F3DAC3E5F3DBC3E6F3005056
:1065C00008E00301E337E391E437E537E637FF0FEF
:1065D000F7D70301110EE26FFF0EE76F1EEC36F0E6
:1065E000005205E044EC3BF0010E006E1200FF0E7D
:1065F0000301EB6F7AEC3BF00050FE0AF8E1030177
:10660000DE6BDF6B020EDF5D02E1000EDE5D14E289
:10661000DE51DC25E06FDF51DD21E16FFF0EEB6F16
:106620007AEC3BF0E0C3E1FFE1C3E2FF00C0E6FF2C
:106630000301DE4BDF2BE6D70301FF0EEB6F7AEC95
:106640003BF0FF0E0301EB6F7AEC3BF044EC3BF0C8
:10665000006A120038EC38F057EC3AF0000E046E85
:10666000000E056E200E066E750E076E17EC2EF0EE
:1066700000C0A4F201C0A5F202C0A6F203C0A7F2B6
:106680000AEC38F057EC3AF0000E046E000E056E7E
:10669000200E066E750E076E17EC2EF000C0A8F2E5
:1066A00001C0A9F202C0AAF203C0ABF2DBEC36F0E3
:1066B000AC0E706F020E716F800E726F780E736F7A
:1066C000000E746F2CC375F32DC376F38D0E776FA8
:1066D000020E786FA4C279F3A5C27AF3A6C27BF347
:1066E000A7C27CF3A8C27DF3A9C27EF3AAC27FF33E
:1066F000ABC280F359EC39F02C4B2D2B120038EC47
:1067000038F057EC3AF0000E046E000E056E200EC5
:10671000066E750E076E17EC2EF000C0A4F201C0D5
:10672000A5F202C0A6F203C0A7F20AEC38F057ECBB
:106730003AF0000E046E000E056E200E066E750E09
:10674000076E17EC2EF000C0A8F201C0A9F202C03B
:10675000AAF203C0ABF2AC0E0301706F020E716FB0
:10676000940E726F780E736F000E746FA4C275F37F
:10677000A5C276F3A6C277F3A7C278F300C079F377
:1067800001C07AF302C07BF303C07CF359EC39F00B
:10679000020EAF6F010EB06FAC0EB16F020EB26F92
:1067A00009EC35F01200010E0301706FE5EC38F0D2
:1067B000000E015C02E1640E005C45E2D9EC39F0A8
:1067C000F00E02013F158D6F8D338D9F8D338D9FA0
:1067D0008D338D9F8D338D9F300E8D270F0E3F157E
:1067E0008E6F300E8E273A0E8F6FF00E3E15906F23
:1067F0009033909F9033909F9033909F9033909FD1
:10680000300E90270F0E3E15916F300E9127926B30
:10681000020E0301AF6F0C0EB06F8D0EB16F020E42
:10682000B26F09EC35F0820E0B6EFF0E0A6E0B2E66
:1068300001D003D00A2EFED7FAD7870E0A6E0A2E91
:10684000FED70000B0D70301DCEC37F012000301E3
:10685000D96B080EDA6F1EC0E9FF0F0EEA6EDA532D
:106860001EE09BEC3BF00000EF8A9BEC3BF0030149
:10687000D95300E0EF8C120EE95EEFAC3DEF34F03F
:10688000EFBAD880EFAAD890D9379BEC3BF06BECED
:106890003BF0120EE926EF9C0301DA07E0D7EF8AFE
:1068A0009BEC3BF00301D85302E06BEC3BF0D8517A
:1068B000D8B45CEF34F0EF9A00009BEC3BF0EF8C27
:1068C000120EE95EEFAC62EF34F0120EE9269BEC9B
:1068D0003BF06BEC3BF0EF9C9BEC3BF06BEC3BF04C
:1068E000EF9AD9C300F012001FC000F020C001F0E1
:1068F00000C01FF001C020F01FC0E9FF20C0EAFF68
:106900000301D85300E0EF96EF94EF9EEF9CEF9ACF
:10691000EF98D8BFEF8ED8BDEF8CD8BBEF8AD8B92F
:10692000EF882150010A02E1EF9402D00301EF84C5
:10693000EF869BEC3BF00301D85300E0EF96EF9419
:10694000EF9EEF9CEF9AEF98D8B7EF8ED8B5EF8C0B
:10695000D8B3EF8AD8B1EF882150010A02E1EF9451
:1069600002D00301EF840301EF869BEC3BF0EF962E
:106970002150010A03E1F1EC3AF002D081EC3BF046
:10698000120030C204F031C205F0000E066E076E30
:1069900004C070F305C071F306C072F307C073F34F
:1069A0000301703770917137723773372AC204F060
:1069B0002BC205F0000E066E076E70C300F071C3A7
:1069C00001F072C302F073C303F06FEC23F000C058
:1069D00022F001C023F02AC204F02BC205F0000E01
:1069E000066E076E70C300F071C301F072C302F04F
:1069F00073C303F06FEC23F008C000F009C001F08E
:106A00000AC002F00BC003F000C024F001C025F062
:106A1000120010D0800E0301AF6F1AD0C00EAF6FFE
:106A200017D0940EAF6F14D0D40EAF6F11D0800E6C
:106A3000AF6F0ED00301AF51010AECE0AF51020A73
:106A4000EDE0AF51030AEDE0AF51040AEDE0EFD7FE
:106A5000B005006EAF51002600C0AFF300C0D8F300
:106A600074EC34F0216A0301B36BB46BB351B125FC
:106A7000E96EB451B221EA6EEECF00F000520EE0A2
:106A8000B351B125E96EB451B221EA6EEECFD8F31D
:106A900074EC34F00301B34BB42BE8D7010E216E34
:106AA0001200BDEC3AF0D00E0301D86F53EC31F078
:106AB0000301D86B53EC31F0BCEC39F0BDEC3AF08B
:106AC000D10E0301D86F53EC31F0010E0301D86FE2
:106AD00027EC34F000C03DF2010E0301D86F27EC23
:106AE00034F000C03EF2010E0301D86F27EC34F001
:106AF00000C03FF2010E0301D86F27EC34F000C054
:106B000040F2010E0301D86F27EC34F000C041F2CF
:106B1000010E0301D86F27EC34F000C042F20301EC
:106B2000D86B27EC34F000C043F2BCEC39F0120013
:106B30002A0E2424E16E000E2520E26EFF0EE66E82
:106B4000010E2424006E000E2520016E2A0E002462
:106B5000E16E000E0120E26EFF0EE66E225026244A
:106B60000301D86F23502720D96F000E2820DA6F39
:106B7000000E2920DB6F2A0EDC6F000EDD6FABEC00
:106B80002EF0225002012C250301D86F2350020160
:106B90002D210301D96F000E02012E210301DA6FAE
:106BA000000E02012F210301DB6F2A0EDC6F000EA5
:106BB000DD6FABEC2EF012000201446B456B466BAF
:106BC000476B486B496B4A6B4B6B4C6B4D6B4E6B19
:106BD0004F6B306B316B346B356B366B376B506B87
:106BE000516B526B536B266A276A286A296A2C6B91
:106BF0002D6B2E6B2F6B226A236A546B556B246AA4
:106C0000256A566B576B2A6B2B6B326B336B586B49
:106C1000596B5A6B5B6B5C6B5D6B396B3A6B3B6BA7
:106C20003C6B386B5E6B5F6B606B616B626B636B55
:106C3000646B656B666B676B686B1200400E0301DB
:106C4000E225EB6F7AEC3BF0E6C3EBF37AEC3BF03A
:106C5000E5C3EBF37AEC3BF0E4C3EBF37AEC3BF007
:106C6000E3C3EBF37AEC3BF0E7C3EBF37AEC3BF0F6
:106C7000FF0E0301EB6F7AEC3BF000C0E8F3030179
:106C8000E96BEA6B0301E851000A16E0E851010ADA
:106C900013E0E9C301F0EAC302F0E94BEA2B4E0E20
:106CA000025C02E1200E015C07E2FF0EEB6F7AEC62
:106CB0003BF000C0E8F3E6D7E8C300F01200010E95
:106CC0000301706F63EC3BF000C095F20050010FC0
:106CD0000201956F010E0301706F95C271F36DECA7
:106CE0003AF0640E046E95C200F0D0EC3AF0300E2B
:106CF000002402019B6F640E046E95C200F0D0EC7C
:106D00003AF008C000F000C04DF34DC395F20A0EF2
:106D1000046E4DC300F0D0EC3AF0300E00240201B6
:106D20009C6F0A0E046E4DC300F0D0EC3AF008C020
:106D300000F0300E002402019D6F120000010C6A69
:106D40000E6A0250D8A4B8EF36F001C002F000C0BD
:106D500001F0006A0E860250D8A4B8EF36F001C0E8
:106D600002F0016A0E960E880250D8B4CAEF36F0CF
:106D70000E50035ED8A4D8A0D0EF36F0D89002BE53
:106D8000D6EF36F0003601360236032EBFEF36F06E
:106D9000D0EF36F0010E0C6E5BEC3BF0DAEF36F024
:106DA000020E0C6E0FEC3BF0DAEF36F0040E0C6EB8
:106DB00087EC3BF0120051EC35F0F00E02013F156C
:106DC0008D6F8D338D9F8D338D9F8D338D9F8D3343
:106DD0008D9F300E8D270F0E3F158E6F300E8E2734
:106DE0003A0E8F6FF00E3E15906F9033909F903358
:106DF000909F9033909F9033909F300E90270F0E6E
:106E00003E15916F300E9127926B020E0301AF6F0A
:106E10000C0EB06F8D0EB16F020EB26F09EC35F033
:106E2000120000010D6A03AE21EF37F0001E011EB3
:106E3000021E031E000E002A012202220322810EDE
:106E40000D2607AE2EEF37F0041E051E061E071E88
:106E5000000E042A0522062207220D2A66EC38F0CD
:106E60000DA044EF37F0001E011E021E031E081E77
:106E7000091E0A1E0B1E000E002A012202220322F6
:106E8000082209220A220B221200000100500402EB
:106E9000F4CF09F0F3CF08F001500502F4CF0BF066
:106EA000F3CF0AF000500502F3500926F4500A22ED
:106EB000E86A0B2201500402F3500926F4500A221A
:106EC000E86A0B2205AE69EF37F000500A5C01500A
:106ED0000B5801AE70EF37F004500A5C05500B58A8
:106EE00008C000F009C001F00AC002F00BC003F0B6
:106EF00012000201A26BA36B800EA319006E800E1C
:106F0000005C02E1080EA25D25E2010E046EA2C241
:106F100000F0A3C201F00450020105E00036009029
:106F20000136FF0FF9D7730E002403014D6F020ED7
:106F300001204E6FA2C270F3E5EC38F04DC3E1FFC3
:106F40004EC3E2FF00C0E6FF01C0E6FF0201A24B14
:106F5000A32BD2D7120000010134083609360450A1
:106F6000085E0550D8A0053C095E003601360F0EBC
:106F70000C6E013408360936045000A0C7EF37F014
:106F8000085E0550D8A0053C095ECCEF37F0082616
:106F90000550D8B0053C0926003601360C2EB9EF55
:106FA00037F000B0DAEF37F0045008260550D8B0BB
:106FB000053C092600001200BDEC3AF0D00E03019A
:106FC000D86F53EC31F00301D86B53EC31F003016F
:106FD000D86B53EC31F03EC2D8F353EC31F03FC2E2
:106FE000D8F353EC31F0070E0301D86F53EC31F0B6
:106FF000200E0301D86F53EC31F0080E0301D86F57
:1070000053EC31F0070E0301D86F53EC31F0BCECB8
:1070100039F0120085C283F286C284F287C285F2FB
:1070200088C286F289C287F28AC288F28BC289F24C
:107030008CC28AF275C28BF276C28CF2020189513F
:107040007525006E8A517621016E87510026885180
:107050000122855100268651012283510026845148
:107060000122050E046E000E056E9EEC39F0120032
:107070006BC269F26CC26AF26DC26BF26EC26CF2E4
:107080006FC26DF270C26EF271C26FF272C270F2B4
:1070900073C271F274C272F202016F517325006EF5
:1070A00070517421016E6D5100266E5101226B5199
:1070B00000266C510122695100266A510122050EF9
:1070C000046E000E056E9EEC39F012000001220ED7
:1070D0000C6E086A096A0A6A0B6A0C06D8B493EF48
:1070E00038F0D8900B320A320932083203320232B9
:1070F00001320032D8A06DEF38F00C06D8B48BEF17
:1071000038F0045008260550092206500A2207507C
:107110000B2272EF38F00450082605500922065061
:107120000A2207500B22120000010B6A0A6A096A40
:1071300000500402F4CF09F0F3CF08F0015005022B
:10714000F4CF0BF0F3CF0AF000500502F3500926FC
:10715000F4500A22E86A0B2201500402F350092677
:10716000F4500A22E86A0B2208C000F009C001F0BE
:107170000AC002F00BC003F01200020E0201305DE3
:10718000046E000E3159056E38C200F0000E016E1B
:10719000026E036E000E066E076E11EC37F000C033
:1071A00034F201C035F202C036F203C037F20201F8
:1071B00039510024346F3A510120356F3B51022080
:1071C000366F3C510320376F1200C26AC00EC212E4
:1071D000C18CC18E70C300F0003600900036009064
:1071E000003600900050C212C28091EC3BF0C28485
:1071F000C2B4FED7080E026EC4CF00F0000E016EBE
:10720000025005E0003600900136FF0FFAD7C35058
:107210000012000E0112C2901200520E0301566FAE
:10722000030E576F4DC370F34EC371F34FC372F328
:1072300050C373F351C374F3560E756F030E766F1C
:1072400075EC11F000C054F301C055F30050030178
:107250004D25E16E01504E21E26EE66A54C300F006
:1072600055C301F012004DC351F34EC352F351C345
:1072700002F052C303F00301514B522B4FC3E9FFFD
:1072800050C3EAFF4F4B502BEECF00F002C0E1FF9E
:1072900003C0E2FF00C0E6FF02C0E9FF03C0EAFF4F
:1072A000EECF00F00052E3E14DC300F04EC301F019
:1072B0001200750E0301836F030E846F70C3AFF36A
:1072C00071C3B0F372C3B1F373C3B2F374C3B3F356
:1072D000830EB46F030EB56F30EC00F000C081F385
:1072E00001C082F3005003017025E16E015071214D
:1072F000E26EE66A81C300F082C301F01200000E64
:10730000156E000E166E000E196E440E0201966F79
:10731000410E976F540E986F410E996F5F0E9A6FE2
:10732000780E9B6F780E9C6F780E9D6F540E9E6F3B
:10733000580E9F6F540EA06FA16B12000001086AD7
:10734000096A100E0C6E0134083609360450085EC6
:107350000550D8A0053C095ED8B0B6EF39F004500E
:1073600008260550D8B0053C0926D89000360136CD
:107370000C2EA3EF39F012001EC0E9FF0F0EEA6ECB
:107380006BEC3BF0EF9A9BEC3BF0EF8C120EE95E5E
:10739000EFACC8EF39F0120EE9269BEC3BF09BEC0A
:1073A0003BF09BEC3BF09BEC3BF0EF8A9BEC3BF023
:1073B000120002013E2B0F0E3E15016E01500A0A0B
:1073C00002E1060E3E27600E3E5D0EE33E6B3F2B54
:1073D0000F0E3F15016E01500A0A02E1060E3F270B
:1073E000240E3F5DD8B03F6B12004DC34FF34EC328
:1073F00050F34FC3E9FF50C3EAFF03014F4B502B3B
:10740000EECF00F00052F5E14D514F5D006E4E5150
:107410005059016E010E005E000E015A120022C08A
:1074200000F023C001F032C204F033C205F094EC46
:1074300038F024C002F025C003F003320232039E6C
:10744000025000240201306F03500120316F1200FE
:10745000000103500718D8A43DEF3AF00250061877
:10746000D8A43DEF3AF001500518D8A43DEF3AF00A
:1074700000500418D8B4D8841200D8941200120016
:10748000949A94969488C66A03014D51C6124F513E
:10749000C6124E51C7124F5305E05051000AD8B4DE
:1074A000C78C03D05053D8A4C78CC68A12000001E1
:1074B0000050086E0150006E016A026A036A0B6A8E
:1074C0000C6A960E036E0A6A00C001F008C000F054
:1074D000086A026A9EEC36F01200A6A202D00000F2
:1074E000FCD7A69C70C3A9FF71C3A8FFA69EA68463
:1074F000F29E550EA76EAA0EA76EA682F28EA694D5
:10750000120000010050086E0150006E0250016E22
:107510000350026E036A0B6A0C6A9E0E036E0A6ABF
:10752000020E0C6EABEC28F01200BDEC3AF0D00E5F
:107530000301D86F53EC31F0070E0301D86F53EC01
:1075400031F0900E0301D86F53EC31F0BCEC39F000
:1075500012004DC3E9FF4EC3EAFF120E03014D2591
:10756000006E00C01EF000C0E9FFEF8AEF8C120E23
:10757000E95EEFACB9EF3AF012001EC0E9FF0F0E62
:10758000EA6EEF8A9BEC3BF0EF8C9BEC3BF06BECF4
:107590003BF0EF9A9BEC3BF06BEC3BF0EF9C120066
:1075A0000001086B080E0C6E003408360450085EAB
:1075B000D8B0DDEF3AF00826D89000360C2ED4EF84
:1075C0003AF01200030170517A0807E3610E705D12
:1075D00004E3010E006EEEEF3AF0006A000E016E59
:1075E0001200080E0B6EFF0E0A6E0B2E01D003D098
:1075F0000A2EFED7FAD71E0E0A6E0A2EFED71200EA
:1076000000010B800BAE0DEF3BF0026A0AAEFF0EDD
:10761000026E016E006E0A360232FF0E1200000189
:107620000B840BAE1BEF3BF0010E036E026A016A86
:10763000006A0A360232FF0E120000010B1E0A1EFB
:10764000091E081E082AD8B4092AD8B40A2AD8B4B0
:107650000B2A120000010B820BAE35EF3BF00368E2
:107660000268016800680A360232FF0E1200030148
:10767000D851390807E3300ED85D04E3010E006EDF
:1076800043EF3BF0006A12001AC0E9FF1BC0EAFF9B
:107690001D50EF12FF0E0301EB6F7AEC3BF012006E
:1076A000030170517A0804E3610E705DD8B0709BDD
:1076B00070C300F012000001026A016A006A086AE1
:1076C000036A000E1200A69C70C3A9FFA69EA680A6
:1076D000A8CF00F01200090E1E5CE16E0F0EE26EE4
:1076E000E79AE79C12001AC0E9FF1BC0EAFF1C5092
:1076F000EF161200EBC3C9FFC7A0FED7C9CF00F039
:107700001200100E0A6E0A2EFED7000012000001B1
:107710000AAE029E000E12000001067EF2EC1DF081
:107720001200070E0A6E0A2EFED7120000010B6A25
:107730000B86FF0E1200000012000000007FCDCC6F
:107740004C7B0AD723786F12037517B75171ACC5FC
:10775000276EBD37066B95BF566777CC2B645F707D
:107760000961FFE65B5D08E53C3C6042221B0000CE
:10777000007F000020820000488500007A880040D9
:107780001C8C0050438F002474928096189620BC65
:107790003E99286B6E9CF90215A0EC782DC1CAF2B7
:1077A00049E2010000000A00000064000000E80354
:1077B000000010270000A086010040420F008096C4
:1077C000980000E1F50500CA9A3B01000000100096
:1077D0000000000100000010000000000100000097
:1077E000100000000001000000100100000008006F
:1077F00000004000000000020000001000000080B7
:107800000000000004000000200000000001000053
:1078100000080000004000000000303132333435F1
:107820003637383941424344454600FF3031323320
:1078300034353637383961626364656600FF0100AC
:107840000A006400E8031027010010000001001086
:107850000100080040000002001000803031323387
:1078600034353637383941424344454600FF3031DC
:10787000323334353637383961626364656600FF08
:1078800025642C25732C25302E33662C25302E3381
:10789000660D0A0025302E33662025302E33660013
:1078A0002530356400FFFFFFFFFFFFFFFFFFFFFFF5
:020000040030CA
:0E000000FFFAFFFEFFFFFBFFFFFFFFFFFFFF0A
:00000001FF
